:020000040800F2
:10000000001800206B6A0008196A0008E16A0008FD
:100010001D6A00081F6A0008216A0008000000002D
:10002000000000000000000000000000236A00083B
:10003000256A000800000000276A0008B1100008C7
:100040002B6A00082D6A00082F6A0008316A000830
:10005000336A0008356A0008376A0008396A000800
:100060003B6A00083D6A00083F6A0008416A0008D0
:10007000436A0008456A0008476A0008496A0008A0
:100080004B6A00084D6A00084F6A0008516A000870
:10009000536A0008556A0008576A0008596A000840
:1000A0005B6A00085D6A00085F6A000825110008A5
:1000B000636A0008656A0008676A0008795E0008DC
:1000C0009023DB05802252049A61024B04221A60BD
:0800D0007047C0467C150020BA
:1000D80033230349034A0A60013B002BFBD17047D5
:0800E80000300040AAAA00004C
:1000F0002E4A91698023DB010B4393619023DB053A
:100100001A682B490A401A601968802292030A4330
:100110001A60284A1168284801401160106880213F
:10012000890101431160596A244801405962586AA3
:100130008021490001435962136A21490B4013622F
:10014000204B214A1360214A1360214B1B68392B35
:1001500027D01CD8132B26D0263B5A1E93415B4236
:100160001C4A13401C4A944663441C4A93818023D2
:100170009B025360002393602C33136013680121AA
:100180000B431360164B802212051A607047603BC8
:100190005A1E93415B42134A1340134A94466344E8
:1001A000E3E7124BE1E7124BDFE7C04600100240E5
:1001B000FFFFEFFF00040048FFEFFFFFFFF0FFFF2E
:1001C000FFFFFFF0FC100020581500205415002000
:1001D00088150020BFFCFFFFE2040000003801404A
:1001E00000E100E019EEFFFF88130000410300006A
:0401F000C40900003E
:1001F40004498022CB691A42FCD080B2014B188595
:080204007047C04600380140BC
:10020C0010B504000D4B1B68002B0AD0023B0222D8
:10021C00934310D00A4B1B68002B0ED005F07AFECE
:10022C000BE0FFF7E1FF064B1B68002B05D020000D
:10023C0005F070FE01E0FFF7D7FF10BD641500203C
:04024C0088140020F2
:1002500010B504003C4B1868C3433C4A1168CA43BC
:100260000140013165D03A4901200860190C394834
:1002700001601B041B0C38480360002902D135497A
:1002800036480860002B02D1334B35491960D1073D
:10029000C91706230B400A3332490B6032490B6001
:1002A00013065B0E31490B6031490B60002C3FD0C7
:1002B00053059B0F2F490B60D10A1F2001400431C9
:1002C0002D4B1960120C2D4B1A602D4B1B68DB4314
:1002D0001A04120C2B490A601B0C03402A4A1360B3
:1002E0002A4B2B4C2B48191904CBD2430A6083426A
:1002F000F9D1294C2948191904CBD2430A60834209
:10030000F9D103F04BFE1F4B1B68002B07D0902345
:10031000DB051B8A5B0502D41A4B00221A600D20F4
:10032000FFF774FF04F0D0F9164B1B68002B05D1C2
:1003300010BD04F00FF8002CE3D1F9E7013B184A97
:10034000136003F039FBF3E700740008047400083D
:100350006C15002014150020701500208304000087
:1003600040570000D8140020AC140020881500204D
:100370005C150020B4140020BC140020B814002028
:10038000087400081015002084150020107400085F
:10039000F893FF17007A00080888FF17008000080C
:0403A000CC14002059
:1003A40010B5114B1B68022219009143012909D091
:1003B400022B0AD0042B0FD00C4A802311680B4364
:1003C400136001E0FFF714FF10BD094B1B68002BFD
:1003D400F2D005F0A3FDF7E7054B1B68002BEBD02B
:1003E40005F0CEFDF0E7C04664150020F0140020AF
:0403F4008814002049
:1003F80010B504003034E4B2392C01D93730C4B216
:100408000F4B1B68002B07D002229343012B0ED001
:100418002000FFF7EBFE10BD2000FFF7E7FE094BB9
:100428001B68002BF7D0200005F076FDF3E7054B9D
:100438001B68002BECD0200005F06EFDEBE7C046F2
:08044800641500208814002057
:10045000F0B5C64600B58CB007A9344B0A0013CBE3
:1004600013C203CB03C201A9314B0A0013CB13C241
:1004700003CB03C2198811809B7893702D4B012206
:100480001A602D4B1B68043B5A4253412B4A1360A0
:1004900004F0FCFE2A4A2B4B1A602B4B98462B4F3C
:1004A000284E2B4D06E02B68002B13D1254B1B68E3
:1004B000002B0FD043461F6034689442F3D0A3054D
:1004C0009B0D244922008B42EDD12E20FFF79EFE8A
:1004D0002200E8E7184B1B68042B13D007A806F08E
:1004E00028FB1B4B1B68002B10D06F20FFF78EFEE4
:1004F0006B20FFF78BFEC82000F0ACF80CB080BC7E
:10050000B846F0BD01A806F014FBEAE76520FFF746
:100510007DFE7220FFF77AFE7220FFF777FE6F20D4
:10052000FFF774FE7220FFF771FEE4E75C6F0008CE
:10053000706F000818150020641500208414002036
:10054000B80B00006015002000300040AAAA00008F
:0805500088140020FF030000E5
:1005580010B5334B1B68002B22D1314B32221A6065
:10056800304B314A1A60314B1B68002B19D0013BC4
:100578002E4A1360002B14D09023DB051B8A9B05A1
:100588000ED52B4B1B68002B0AD02A4B1B68002B5F
:1005980006D0294B1B685A1C132B08D0264B1A600F
:1005A80010BD9023DB05802252009A61E4E7224BBC
:1005B80000221A60214B1B68002B09D1204B1B68B5
:1005C800002BEDD1FFF740FF0D20FFF71BFEE7E7FB
:1005D8001C4B1B68042B0FD01B4B1B68012BDFD156
:1005E80004F036FD184B00221A60FA20400000F093
:1005F8002DF8FFF729FFD3E7134B1B68002BCFD14A
:1006080004F026FD104B01221A60FA20400000F089
:100618001DF8FFF719FF0B4B1B68042BC0D0DBE755
:100628006815002000300040AAAA00007C150020B0
:100638001415002070150020641400208814002070
:0C06480018150020641500208414002008
:1006540010B5054B1860002805D01C00FFF77AFF81
:0C0664002368002BFAD110BD8015002087
:10067000F8B5D1490122CB681A42FCD1CE4B1B6997
:100680001B0604D5CC4BCD4A5A60CD4A5A60CA4BA2
:100690001A6902210A431A61CA4A5A611A693E312B
:1006A0000A431A6119000122CB681A42FCD1C24BDD
:1006B000DB689B0604D5C04AD36820210B43D36076
:1006C000BD4B1A6902218A431A611A6901390A432A
:1006D0001A61BD4B1B68DB43BA4A1380B64901223D
:1006E000CB681A42FCD1B44BDB689B0604D5B24AF6
:1006F000D36820210B43D360B44B1B68DB43B44A5F
:100700001380AD490122CB681A42FCD1AA4BDB68A9
:100710009B0604D5A84AD36820210B43D360AD4B78
:100720001B685B00FF221A40AB4B1B680A3B591E3B
:100730008B411A43A94B1B685B02C021C9000B40C7
:100740001A43A74B1B68043BDB061B0C1343DB431C
:10075000A44A138098490122CB681A42FCD1964BD7
:10076000DB689B0604D5944AD36820210B43D360F1
:100770009D4B1B68DB439D4A13808F490122CB6848
:100780001A42FCD18C4BDB689B0604D58A4AD3689D
:1007900020210B43D360964B1B68DB43954A1380A3
:1007A00085490122CB681A42FCD1834BDB689B064A
:1007B00004D5814AD36820210B43D3608E4B1B683C
:1007C000DB438E4A13807C490122CB681A42FCD15C
:1007D000794BDB689B0604D5774AD36820210B430D
:1007E000D360874B1B68DB43864A13807249012222
:1007F000CB681A42FCD1704BDB689B0604D56E4A6D
:10080000D36820210B43D3607F4B1B68DB437F4AB7
:10081000138069490122CB681A42FCD1664BDB6820
:100820009B0604D5644AD36820210B43D3607848E3
:10083000784C241A604B01222025774F02E00430C7
:10084000B8421AD006190168C9433180D9680A42F2
:10085000FCD1D9680D4202D0D9682943D96001681A
:10086000C943090C7180D9680A42FCD1D9680D428C
:10087000E5D0D9682943D960E1E74F4B1A690121D6
:100880008A431A61654A664911601A6902210A435E
:100890001A61644A5A611A693E310A431A611900A1
:1008A0000122CB681A42FCD1434BDB689B0604D57E
:1008B000414AD36820210B43D3603F4B1A69022180
:1008C0008A431A611A6901390A431A61524801229E
:1008D0002025554F02E00430B8421AD006190168AD
:1008E000C9433180D9680A42FCD1D9680D4202D08F
:1008F000D9682943D9600168C943090C7180D96856
:100900000A42FCD1D9680D42E5D0D9682943D960A3
:10091000E1E74648464C241A274B01222025454F43
:1009200002E00430B84219D006190168C943318089
:10093000D9680A42FCD1D9680D4202D0D96829434E
:10094000D9604188C9437180D9680A42FCD1D9680D
:100950000D42E6D0D9682943D960E2E7164B1A69FF
:1009600001218A431A612D4A2D4911601A69022119
:100970000A431A61304A5A611A693E310A431A61C0
:1009800019000122CB681A42FCD10B4BDB689B0695
:1009900004D5094AD36820210B43D360064B1A695A
:1009A00002218A431A611A6901390A431A61012234
:1009B0002025224F47E0C046002002402301674522
:1009C000AB89EFCD007400087015002014150020CD
:1009D0000274000888150020D8140020B4140020E8
:1009E000BC14002004740008B81400200674000829
:1009F0001015002008740008841500200A740008EF
:100A0000D41400200C740008D01400200E740008C8
:100A10000808002010740008F80B00200030004087
:100A2000AAAA000000780008F80D002008020020A3
:100A3000007A000808040020007C00080808002054
:100A40000430B84219D006190168C9433180D96809
:100A50000A42FCD1D9680D4202D0D9682943D96035
:100A60004188C9437180D9680A42FCD1D9680D42D6
:100A7000E6D0D9682943D960E2E7064B1A6901211B
:100A80008A431A611A697F310A431A610A20FFF703
:080A9000E1FDF8BD0020024069
:100A980070B5041E00DA9CE0092C00D893E0632CA2
:100AA80000D881E0FA239B009C426ED3534B9C42B2
:100AB8005AD9534B9C4248D9524B9C4236D9524B37
:100AC8009C4224D9514B9C4212D9514B9C4200D98B
:100AD80084E05049200006F018FB05004D4920002D
:100AE80006F001FA0C0028003030C0B2FFF78AFB8C
:100AF8004949200006F009FB05004749200006F097
:100B0800F2F90C0028003030C0B2FFF77BFB4349F4
:100B1800200006F0FAFA05004049200006F0E3F943
:100B28000C0028003030C0B2FFF76CFB3C492000B5
:100B380006F0EBFA05003A49200006F0D4F90C005B
:100B480028003030C0B2FFF75DFB3649200006F0C0
:100B5800DCFA05003349200006F0C5F90C0028002E
:100B68003030C0B2FFF74EFBFA218900200006F0B2
:100B7800CCFA0500FA218900200006F0B4F90C002F
:100B880028003030C0B2FFF73DFB6421200006F09A
:100B9800BCFA05006421200006F0A5F90C00280025
:100BA8003030C0B2FFF72EFB0A21200006F0ADFA64
:100BB80005000A21200006F096F90C0028003030C4
:100BC800C0B2FFF71FFB20003030C0B2FFF71AFB9E
:100BD80070BD2D20FFF716FB64425DE71249200027
:100BE80006F093FA05001049200006F07CF90C0085
:100BF80028003030C0B2FFF705FB6AE70F27000076
:100C08009F8601003F420F007F969800FFE0F505A0
:100C1800FFC99A3B00E1F5058096980040420F0015
:0C0C2800A08601001027000000CA9A3BC3
:100C340070B58CB006AD124B2A0013CB13C213CB84
:100C440013C26C460F4B220043CB43C243CB43C277
:100C54000D20FFF7D9FA280005F069FF3520FFF7CA
:100C6400D3FA2E20FFF7D0FA2420FFF713FF200039
:100C740005F05DFF0D20FFF7C7FA0CB070BDC0464C
:080C8400F46200080C63000893
:100C8C0010B5584B5969802292020A435A6159692E
:100C9C008022D2020A435A619022D20500231360AB
:100CAC0051490B605148D0605148C860D068514CD4
:100CBC002040D060116821401160106880214902E9
:100CCC00014311608021490091614B4ACE3911607A
:100CDC004A4A13604A4A13604A4A13604A4A4B49CB
:100CEC0011604B4A4B4911604B4A13604B4A1360DD
:100CFC004B4A13600A224B490A604B490A604B4A23
:100D0C0013600B224A490A604A490A604A4A136036
:100D1C004A4A13604A4A13604A4B4B4A1A604B4B7F
:100D2C001868FA21890006F0EEF9013880235B047B
:100D3C0098420DD2464A50604648036A1B021B0A71
:100D4C00C02109060B430362002393600733136031
:100D5C000A20FFF779FC404C404B2360404BA360CA
:100D6C000220FFF771FC022363600220FFF76CFC8A
:100D7C003C4B23600020FFF765FA0220FFF764FC70
:100D8C00FFF7B0F90220FFF75FFCFFF74DFF0220E1
:100D9C00FFF75AFC344B00221A609023DB051B8AA8
:100DAC009B0507D5184B1B68002B03D0184B1B68F1
:100DBC00934213D12D4805F0B6FE0D20FFF714FA1F
:100DCC000120FFF73FFA2A4C03F04AF902F01EF813
:100DDC002368002BF8D002F04DFEF5E7FFF732FB4D
:100DEC00EEE7C0460010024000040048AAAA0AA47C
:100DFC00AAAAAAAAFFFFFCFF681500207C150020F8
:100E0C0080150020601500201415002083040000BC
:100E1C007015002040570000841400201815002085
:100E2C006C150020D8140020AC1400206415002090
:100E3C00881500205C1500208415002078150020F2
:100E4C0074150020C4140020A1B0B91204020020B3
:100E5C0010E000E000ED00E00030004055550000CF
:100E6C00FFFF0000CCCC000088140020886F000825
:040E7C00A01400209E
:100E800010B5FFF769FB0F4B1B680F4A12689342BE
:100E900016D05A1C0B490A601B78802000021843A8
:100EA0000A4B1B689A4208D09023DB05802252042B
:100EB0009A61074B04221A6010BD064A0A60F3E7E4
:100EC0000020F9E7541500205815002000020020EA
:080ED0007C150020FC1000203D
:100ED80010B50E4B1B68002B0AD10D4B1B68002B5D
:100EE80003D004F0FBFD002801D1FFF7C5FF10BDBA
:100EF800023B0222934306D0054B1B68002BF6D019
:100F080004F0ECFDF3E7FFF7B7FFF0E76415002006
:040F18008814002019
:100F1C0010B57F2845D90300F03B0D2B03D8484A68
:100F2C00DA40D30716D4F6281CD0F7281AD8454B2C
:100F3C001A680F230340511E8B4201D0002A28D17E
:100F4C00414B1860F0231840404B1860404B012275
:100F5C001A6006E000233E4A13603B4A13603B4A8A
:100F6C00136010BD3B4B1B68990000043A4A885033
:100F7C005A1C1F2B09D0374B1A600023344A1360BC
:100F8C00314A1360314A1360EBE7324B00221A608E
:100F9C00F3E700232E4A13602B4A13602B4A13608D
:100FAC00DFE72B4B1B68002B19D0012B1ED0022B1B
:100FBC00D7D1284B1A689400234B1B681B04274974
:100FCC00096809020B431843234BE050531C1F2A9A
:100FDC0031D0204A13601E4B01221A60C1E71A4A15
:100FEC0013601A4A13601D4A1360BAE71B4B186052
:100FFC00164B1B6810229343C02B09D0124B1B6855
:10100C000E3A9343F12B03D0114B02221A60A8E73E
:10101C00104B1A6891000C4B1B681B0418430E4BA9
:10102C00C850531C1F2A02D00A4A136099E7094B77
:10103C0000221A6095E7074B00221A60CBE7C046E6
:10104C00B122000084150020601400206C140020D4
:10105C0068140020781500208C1200208C150020BC
:10106C0010B5FFF773FA0C4B1B680C4A12689342CD
:10107C000FD099000A4A8A588020000610435A1C47
:10108C001F2B02D0044B1A6010BD034B00221A60B8
:10109C00FAE70020F8E7C046741500207815002008
:0410AC008C12002082
:1010B000164B1B68002B02D0013B144A1360144BE3
:1010C0001B68002B02D0013B114A1360114B1B68B7
:1010D000002B02D0013B0F4A13600F4B1B68002B03
:1010E00002D0013B0C4A13600C4B1B68002B02D052
:1010F000013B0A4A13600A490A6853035A40530CD9
:1011000053405A0153400B607047C0466815002099
:101110008015002060150020E4140020B014002089
:04112000C4140020D3
:1011240010B51B4BDB699B062CD5194B9B8C9BB2D2
:10113400184A126802218A43012A19D0FF221A4050
:10114400022A0FD0042A10D0134A11680B701368B6
:1011540001331360114A1268934213D10E4B104AA3
:101164001A600FE00F4A1160EEE700F063FD09E03A
:10117400094A11680B70136801331360074A126837
:10118400934200D010BD044B054A1A60FAE7C046EA
:10119400003801406415002058150020000200208A
:0811A400FC100020A41400203F
:1011AC00024A202311680B4313607047F01400208F
:1011BC00064A1368043B1360054A0C32934204D26E
:1011CC00044A042311680B4313607047C0140020B9
:0811DC0010140020F0140020A3
:1011E400084B1A68111D1960074B4033994202D20B
:1011F400136853607047054A042311680B43136056
:10120400F8E7C046C014002010140020F014002099
:10121400044B19680A1F1068096811601B6818607C
:081224007047C046C014002011
:10122C00034A1368191D11601A1F12685A6070471F
:04123C00C0140020BA
:10124000074A1368190008390868043B1B680B60DB
:101250001368191F1B680B60136818607047C0463D
:04126000C014002096
:10126400074A13681968181F006818601368181F64
:10127400083B1B6803601368083B19607047C0464D
:04128400C014002072
:101288000C4B19680A680C4BCB1A9B109B1A042B41
:1012980006D4002A0AD092008A1A13680B60704795
:1012A800064A042311680B431360F8E70439014B1D
:1012B8001960F4E7C014002010140020F014002076
:1012C80030B5144B1A681168134BD31A9B105B1A6C
:1012D800042B19D4043A0F4B1A60012913D901239E
:1012E8005B1A9B009D580222521A9200094C2368EF
:1012F80098589B18043B1860013904320029F6D12C
:10130800044B1B681D6030BD044A042311680B435D
:101318001360F8E7C014002010140020F014002017
:10132800F0B5144B1A681568134BD31A9B105B1B46
:10133800042B19D4043A17680E4B1A60012D12D9E0
:101348006E1E0422524200211C00236898589B18E4
:1013580058600131043AB142F7D101235D1B054BB6
:101368001B68AD00EF50F0BD044A042311680B431D
:101378001360F8E7C014002010140020F0140020B7
:10138800054B1A68111F12680868844662440A608F
:0C1398001A68043A1A607047C014002064
:1013A400024B1A681368013313607047C01400209D
:1013B400054B1A68111F12680868821A0A601A68B5
:0C13C400043A1A607047C046C0140020B4
:1013D000024B1A681368013B13607047C014002069
:1013E000044B1A681368002B00DB70475B421360E4
:0813F000FBE7C046C014002019
:1013F80010B50F4B1B681A68D117501848401F28A2
:1014080009DC191F0A4C2160002A0BDB0B00096854
:101418009140196010BD074A8023DB0011680B4317
:101428001360F7E7043B1A68C2401A60F2E7C04647
:08143800C0140020F014002094
:10144000054B1A68111F1268086802400A601A6882
:0C145000043A1A607047C046C014002027
:10145C00054B1A68111F1268086802430A601A6863
:0C146C00043A1A607047C046C01400200B
:10147800054B1A68111F1268086842400A601A680A
:0C148800043A1A607047C046C0140020EF
:10149400024B1A681368DB4313607047C0140020C2
:1014A400024B1A6813685B4213607047C014002033
:1014B400054B1A68111F1268086842430A601A68CB
:0C14C400043A1A607047C046C0140020B3
:1014D00010B50B4B1C682168002909D0043C20681A
:1014E00005F0F9FD2060064A1368043B136010BD47
:1014F000044A80231B0111680B431360F7E7C046C1
:08150000C0140020F0140020CB
:1015080010B50B4B1C68216800290AD0221F1068EF
:10151800083C23685843064B1C6005F0D8FD206042
:1015280010BD044A80231B0111680B431360F7E7C1
:08153800C0140020F014002093
:1015400010B50B4B1C682168002909D0043C2068A9
:1015500005F0F3FD2160064A1368043B136010BDDB
:10156000044A80231B0111680B431360F7E7C04650
:08157000C0140020F01400205B
:1015780070B50D4B1C682568002D0ED0043C2668FC
:101588002900300005F0D5FD2160074B1C682900B3
:10159800300005F09CFD206070BD044A80231B01CB
:1015A80011680B431360F7E7C0140020F014002003
:1015B800034A1368191D1160024A12685A6070477D
:0815C800C0140020C41400202F
:1015D000064A1368191F1B6808681B1A58424341C2
:1015E0000B601368043B13607047C046C0140020B2
:1015F000064A1368191F1B6808681B1A581E834186
:101600000B601368043B13607047C046C014002091
:10161000034B1A6811684B424B4113607047C04638
:04162000C0140020D2
:10162400074B1A68131F012112681868904200DCE6
:1016340000211960024A1368043B13607047C046D6
:04164400C0140020AE
:1016480030B5074B1A68111F10680A68D217C40F03
:101658000D68854262410A601A68043A1A6030BD12
:04166800C01400208A
:10166C00074B1A68131F012112681868904200DB9F
:10167C0000211960024A1368043B13607047C0468E
:04168C00C014002066
:10169000064A1368191F1B68086884469C459B41CD
:1016A0005B420B601368043B13607047C01400205A
:1016B00030B5074B1A68111F08681468C20FE51788
:1016C00084426A410A601A68043A1A6030BDC04612
:0416D000C014002022
:1016D4000B4B1B681A680B498A420AD30A498A428F
:1016E40007D8043B1B681360054A1368083B136062
:1016F40004E0064A202311680B4313607047C04678
:10170400C014002008080020F80D0020F014002068
:10171400084B1A68136808498B4205D307498B4262
:1017240002D81B68136004E0054A202311680B43A8
:1017340013607047C014002008080020F80D002032
:04174400F01400207D
:10174800044B0A221A60044B1B68002B01D1034B7F
:101758001A607047AC140020F4140020D81400203C
:10176800044B10221A60044B1B68002B01D1034B59
:101778001A607047AC140020F4140020D81400201C
:1017880006490A681368043A0A60002B05D0044920
:10179800044A0A60013B002BFBD17047C0140020AB
:0817A80000300040AAAA000075
:1017B00004490B6864221868424303480260043BF2
:0C17C0000B607047C0140020B014002023
:1017CC0010B5054B1C68221D1A60044B1868642167
:1017DC0005F099FC606010BDC0140020B01400200E
:1017EC0030B5094B1B68013B08495B181B041C0CEA
:1017FC00074802681B0E15684B5513689C466144DC
:10180C004C70043A026030BD001500200802002024
:04181C00C0140020D4
:10182000044B1A68111D1960034B1B68043B1B68AD
:0C18300053607047C0140020C814002052
:10183C00024B1B681A68024B1A607047C8140020D0
:04184C00EC14002078
:10185000064B1B681A68002A04D1054A12681168F1
:10186000044A1160043B014A13607047C014002011
:08187000C8140020EC14002054
:10187800154B1B68154A19681160154A934218D907
:10188800144A1268022A07D0043B0F4A1360124A0E
:101898001368013B136070470F4A11680F4A1268BA
:1018A8009142F1D10D4A002111600A4A03311160B9
:1018B800EAE7064B00221A60064B1B68022BEAD1A6
:1018C800044B03321A60E6E7C8140020EC14002029
:1018D800C0130020F4010020E01400200C150020A3
:1018E800054B00221A605A609A6018000C300349B0
:1018F8000860DA607047C04610140020C014002049
:0C190800014B03221A607047F40100201C
:0C191400014B01221A607047F401002012
:0C192000014B00221A607047F401002007
:10192C0030B50D4B1C68221D1A600C490B685A1CF3
:10193C000A60587800069A1C0A609A7812040243CE
:10194C00D81C0860D87800021D1D0D601B7913434C
:10195C000343636030BDC046C0140020EC1400206B
:10196C00054A1368191D116004490A68501C086067
:10197C0052785A607047C046C0140020EC14002006
:10198C00074B19680A1D1A60064A1368581C106028
:10199C005A781201044B9B189B684B607047C046E9
:0C19AC00C0140020EC14002008080020EB
:1019B800074B1A68511C19600648036851780901D9
:1019C800054A521819689160043B03607047C04685
:0C19D800EC140020C014002008080020BF
:1019E400074B1A68511C196051780902901C186041
:1019F40092781143802292050A431A607047C046C8
:041A0400EC140020BE
:101A080010B5094B1868021D1A6008490B685A1C62
:101A18000A605A7812029C1C0C609B781A43802337
:101A28009B051343436010BDC8140020EC1400202C
:101A3800084B094A1A60094B1A68511C19605178F9
:101A48000902901C186092781143802292050A437B
:101A58001A60704700300040AAAA0000EC14002069
:101A680010B5094B1B681A68023A80239B0513437B
:101A78001A78722A03D1013B044A136010BD034A45
:101A88001360FFF7D5FFF9E7C8140020EC14002015
:101A980010B50A4B1B681B68002B0CD0084A13684A
:101AA800043B1360074A136803331360034A13683F
:101AB800043B136010BDFFF7BBFFF7E7C01400201D
:081AC800C8140020EC140020FA
:101AD00010B50A4B1B681B68002B0CD1084A136811
:101AE000043B1360074A136803331360034A136807
:101AF000043B136010BDFFF79FFFF7E7C014002001
:081B0000C8140020EC140020C1
:101B080010B5104B1A681100103119600E490B6896
:101B1800180008380068D060181F006890601868BE
:101B280050600C3B0B6009480368591C01605978E8
:101B380009029C1C04609B78194380239B050B4376
:101B4800136110BDC8140020C0140020EC1400203C
:101B580010B5254B1B681A1F126819000839086848
:101B68000C3B19685318214A214C146000291DDBCD
:101B7800984212DD1C4A1268043A13601D4B1A6819
:101B8800511C196051780902901C18609278114311
:101B9800802292050A431A6010BD134A1368103B4D
:101BA8001360144A136803331360F5E7984212DA96
:101BB8000D4A1268043A13600E4B1A68511C1960DA
:101BC80051780902901C186092781143802292057E
:101BD8000A431A60E0E7044A1368103B1360054A99
:101BE800136803331360D7E7C8140020003000409F
:081BF800AAAA0000EC14002071
:101C0000024A1368043B13607047C046C8140020A2
:101C1000024A1368103B13607047C046C814002086
:101C200010B5044C23681878FEF7F0FA2368043BDB
:081C3000236010BDC014002068
:101C380000B583B06A46094B03CB03C2084B1B6847
:101C4800002B01D003B000BD684604F06EFF044BC2
:101C580001221A60034B00221A60F3E7246300088C
:081C6800F4010020A414002087
:101C700000B58FB036220F49684605F064F90E4B67
:101C80001B681B68102B0DD80C4A1360002B05D065
:101C9000094A1368043B13600FB000BD684604F0A6
:101CA00048FFF5E7064A8023DB0011680B43136009
:101CB000F2E7C046FC6A0008C0140020841500202A
:041CC000F0140020FC
:101CC40010B5114B1B68002B12D0104B1B78002B46
:101CD4000ED00F4B1B68002B15D00E4A1368191D2C
:101CE40011600D4A12785A60094B00221A600AE00A
:101CF400FFF7F0F80028FBD0064B1A68111D196095
:101D0400FF231840506010BDF40100209F150020EF
:0C1D1400A8140020C01400209E15002020
:101D200010B50E4B1B68102B08D00D4B1B681868A4
:101D3000E0231B06C2180B4B9A420CD8084B1B68B9
:101D4000186805F0BCF92020FEF760FA044A136811
:101D5000043B136010BDFEF79FFEF4E7AC140020B7
:081D6000C0140020FF0B063047
:101D680010B5064C2368186805F0A5F92020FEF781
:101D780049FA2368043B236010BDC046C014002004
:101D8800F0B587B003AA2A4B13CB13C2294B1A68A4
:101D980001929A8801AB9A805B20FEF733FA264BB2
:101DA8001B68264A0C3293420DD0244A0C329342C7
:101DB8000DD3224A0C32934216D9204C10340425F4
:101DC8001E4F160024E001A804F0AFFE0CE003A8A3
:101DD80004F0ABFE194B00221A605A609A60180092
:101DE8000C3015490860DA605D20FEF70BFA2020F8
:101DF800FEF708FA07B0F0BD206805F05CF920206E
:101E0800FEF700FA01350C4B1B680434B342EBD9DA
:101E1800DB1B9B10AB42E7D32020FEF7F3F9084BFE
:101E28001B68102BE8D02068FEF732FEE7E7C046B3
:101E38004C6B0008586B0008C014002010140020D8
:041E4800AC140020B6
:101E4C00F0B5D6464F464646C0B584B001AA394BCC
:101E5C0003CB03C21B7813702020FEF7D1F9364B4D
:101E6C001B68002B5BD0354D00270026C0231B05BB
:101E7C009946334B9A46304B984616E02020FEF795
:101E8C00BFF914E06B684A46134221D12020FEF7BB
:101E9C00B7F92020FEF7B4F901360137052F34D8F5
:101EAC00103543461B68B34237D9092EE6D93000AA
:101EBC00FEF7ECFD3A20FEF7A3F92C00083C207845
:101ECC000028DFD0FEF79CF90134AC42F7D1D9E7FA
:101EDC0001A804F028FE53461B68102B11D028686B
:101EEC00FEF7D4FD2020FEF78BF94020FEF788F991
:101EFC002804000C05F0DDF82920FEF781F90237E3
:101F0C00C4E7286805F0D5F8ECE70D20FEF778F962
:101F1C002020FEF775F90027C2E7002F05D104B089
:101F2C00E0BCBA46B146A846F0BD0D20FEF768F9F4
:101F3C00F5E7C046446E0008DC14002010080020B1
:041F4C00AC140020B1
:101F500010B5044C2368186804F01DFE2368043B88
:081F6000236010BDC014002035
:101F680010B5044C23681878FEF718FA2368043B68
:081F7800236010BDC01400201D
:101F8000F8B50D4A13681F68043B1360002F0CD08E
:101F90000124E41BA4003D0016003368185DFEF721
:101FA00001FA013D0434002DF7D1034BBF001A683C
:0C1FB000D71B1F60F8BDC046C014002005
:101FBC00F0B5C64600B582B06846214B020012CB84
:101FCC0012C204F0B0FD0D20FEF71AF91D4DF823D6
:101FDC009B009846A8440026012723E0FEF710F941
:101FEC000134285D0028F9D1062C05D82020FEF7F5
:101FFC0007F90134072CF9D12320FEF701F9380039
:10200C0004F0A7FD2020FEF7FBF82020FEF7F8F8DF
:10201C002020FEF7F5F801370136052E07D00835DC
:10202C00A84509D02020FEF7EBF80024D9E70D20B5
:10203C00FEF7E6F80026F2E702B080BCB846F0BD29
:08204C002C6300081C6600086B
:1020540070B5FEF73FFF041E00D1D8E0C0B2704B4C
:102064001B68002B08D06F4B1B78002B04D06E4BE1
:1020740018706E4B01221A600A2800D1C4E00228AD
:1020840000D8C3E0674B1B78002B08D109281FD068
:10209400674A12683F2A02D9202800D19EE02828E6
:1020A40018D02F2840D01B2868D10024002B00D141
:1020B400ADE00E38FEF7A8F85D4B1A685D4B2021A1
:1020C40099549B18002159705B4B1A6002349EE0AE
:1020D4001730DDE7594B1C68002C01D0002496E032
:1020E400FEF792F8FEF7F6FE0028FBD0C0B22028D7
:1020F4000BD04F490B684F4A2825D554D21850703D
:1021040002330B60FEF780F881E0494B1B68013312
:102114004A4A13601838FEF777F82020FEF774F85F
:102124000820FEF771F872E0444B1C68002C01D0C3
:1021340000246CE0FEF768F8FEF7CCFE0028FBD024
:10214400C0B22F280BD03A490B683A4A2F25D554F0
:10215400D218507002330B60FEF756F857E0344B38
:102164001B680133354A13602738FEF74DF82020E9
:10217400FEF74AF80820FEF747F848E0092848D057
:10218400122848D0082817D12C4B1D680024002D94
:102194003DD1274B1C68002C39D0013C1C60254BD9
:1021A40020221A55FEF730F82020FEF72DF80820DB
:1021B400FEF72AF82C002AE00D2817D11C4B1B68C7
:1021C400002B0BD11A4B1A681A4B202199549B18D7
:1021D40000215970184B1A60012418E0174B1B6832
:1021E400012BEFD00D20FEF70FF8EBE7134B1C6823
:1021F400002C12D10E4D0F4B2A689854FEF704F8A8
:102204002B6801332B6002E0002400E0002420004E
:1022140070BD0324FBE70424F9E70024F7E7C04674
:10222400F40100209F1500209E150020A814002012
:102234009C1400200C130020A0140020F81400208B
:1022440010B5154B1968154B5A5C202A09D14B1C43
:102254001248013819000133C25C202AFAD00E4B0F
:1022640019600023002A10D00C4840180C4CC25CA2
:10227400202A03D01A5501330F2BF8D1084A002025
:10228400D0545B18074A136010BD054B00221A7026
:10229400044B1960F8E7C046941400200C13002086
:0822A400701300209C140020BF
:1022AC00F0B5DE46474680B587B00E0002AA002482
:1022BC0005E0002B1BD001340132102C08D0035D3B
:1022CC001370190061391929F3D8203B1370F2E708
:1022DC00002302AAD37313782D2B0ED1254B002289
:1022EC001A6001239B460127012C0FD82CE00023F8
:1022FC0002AAD37313782D2B2CD01E4B00221A60FC
:10230C0000239B4600270120002C2DD0194B1D6863
:10231C00B84602AB9C46E044002301934346187830
:10232C00310004F054FC431C18D075432D180137B0
:10233C0001239C46E0440193A742EFD30D4B1D6053
:10234C0001205B46002B0FD00A4A13685B421360D6
:10235C00012009E00020012CC0D105E0019B002BDD
:10236C0001D0044B1D60002007B0C0BCBB46B0467A
:08237C00F0BDC04698140020DA
:1023840010B5344B187800285AD000233149013352
:102394005A5C002AFBD12D280FD0302829D12D4A90
:1023A400527820218A43582A11D02B4A11681029C7
:1023B4003AD1082B48D900204BE0012B3AD0264AC9
:1023C400116810292AD00B2B3ED9002041E0214A64
:1023D40092782D2A09D00A2B2ED81E4810210230BB
:1023E400FFF762FF431E984133E00B2BF5D9002021
:1023F4002FE02528D9D1174A52782D2A09D00B2B42
:102404001CD814480A210130FFF74EFF431E98419F
:102414001FE00C2BF5D900201BE000232D28C8D188
:10242400092B11D9002014E02D28CCD000200A2B30
:102434000FD809E000200CE000200AE0002008E0AA
:10244400054B19681029E8D00248FFF72DFF431EF9
:0C245400984110BD70130020AC14002053
:10246000F0B51A4C00251A4E0021635C8A5D1800F5
:10247000613819280DD8203BDBB2100061381928CB
:1024800011D8203AD2B2934219D101310829ECD1A6
:1024900015E01000613819280DD918002038471EA2
:1024A000B84140420340934209D1002AEDD1094B83
:1024B0001D600120F0BD203AD2B2202BE3D10135BE
:1024C00008347D2DD0D10020F4E7C0461466000802
:0824D00070130020CC14002061
:1024D80070B51A4B1B78002B29D0194A00231E000F
:1024E800013310321100103909780029F7D1731C13
:1024F8001FD03301114C1C19124D16E08B4211D11B
:1025080000290BD00132082A0CD0A15C535D1800B9
:1025180061381928F2D8203BDBB2EFE70A4B1E607E
:10252800012070BD103C013E05D30022EDE70020DC
:10253800F7E70020F5E70020F3E7C0460808002089
:0C2548001808002070130020CC140020A4
:1025540010B50F4B1A680F4B1A60FFF771FEFFF7A7
:10256400B9FF002805D00C4B1B6801330B4A1360DC
:1025740010BD0B4B1B78302B05D00A4A2123116860
:102584000B431360F4E7054B00221A60F0E7C046E2
:102594009C14002094140020CC140020101500205A
:0825A40070130020F014002068
:1025AC00074A13680749C85401331360064A93421B
:1025BC0004D9064A202311680B4313607047C046A8
:1025CC000015002008020020FE050000F014002079
:1025DC0010B5144B18688200134BD3581A030AD445
:1025EC00124A1268002A13D19B030BD48000104BA3
:1025FC00C358984705E00F4A80239B0011680B4392
:10260C00136010BD0B4A082311680B431360F8E7E5
:10261C00DB0304D58000064BC3589847F1E7FFF75E
:10262C00BFFFEEE7CC14002020640008F414002057
:08263C0000000020F014002052
:1026440070B594B00CA9414B0A0013CB13C213CB41
:1026540013C203CB03C205A93D4B0A0013CB13C21B
:1026640013CB13C21B7813706A463A4B13CB13C2B5
:1026740011001A680A601B790B71374B1B68522BC7
:1026840009D95224354E344DA05DFDF7BDFD01340A
:102694002B68A342F8D85223314A1360314A0021EF
:1026A4001160314A13602E4D304E03E02C4B1A68F2
:1026B4002D4B1A60284C2B682268934234D2FFF7C2
:1026C400BFFD3378002BF6D0FFF75AFE00280BD05D
:1026D400274B1A68274B1A60274B1B78002BE5D031
:1026E400264B01221A60E1E7FFF7B8FE002811D05B
:1026F400234B1B689B00234A9B585B0321D5FFF7A0
:102704006BFF214B1B68002B08D1154B1A68164B25
:102714001A60CFE70CA804F00AFA05E01A4B00226D
:102724001A60684604F003FA0D20FDF76DFD52238C
:10273400094A13600A4A13600A4B00221A6014B053
:1027440070BD05A804F0F3F9EEE7C0465C6E00081E
:102754007C6E0008986E0008A01400200C13002062
:102764009C140020F81400209414002070130020FE
:1027740098140020041500209F150020081500203F
:0C278400CC14002020640008F014002099
:1027900070B56C20FFF70AFF0C4D2C68FF20FFF787
:1027A00005FFFF20FFF702FF2B68013B084A9B183B
:1027B0001B04180C074909681B0E0D6853550B685C
:1027C0009C46624450700C6070BDC04600150020ED
:0827D00008020020C0140020E3
:1027D80010B56D20FFF7E6FE064A1368191D116053
:1027E800054A12685A60FF20FFF7DCFEFF20FFF75A
:0C27F800D9FE10BDC01400200015002008
:1028040010B57120FFF7D0FE064A1368191D116038
:10281400054A12685A60FF20FFF7C6FEFF20FFF743
:0C282400C3FE10BDC014002000150020F1
:10283000F8B57220FFF7BAFE104E33681D680135F7
:102840000F4C2D19280AFF273840FFF7AFFE38003C
:102850002840FFF7ABFE0B4B1B68013B1B1932688E
:10286000190A106821541268A41863707420FFF7C5
:102870009DFE3368043B3360F8BDC046C0140020A1
:082880000802002000150020F1
:1028880010B51F4B1B68002B17D11E4B1B681E4A27
:10289800196811601D4A93422ED91D4A1268022AEE
:1028A8001DD0043B174A13601A4A1368013B136092
:1028B800194B1A68194B1A6010BD6120FFF772FE98
:1028C80000220F4B1A6016490B6801330B601B017D
:1028D80014495A54144B1A68144B1A60E8E70D4A05
:1028E8001168134A12689142DBD1114A0021116024
:1028F800074A03311160D4E7034B00221A60D7E777
:10290800F4140020C8140020EC140020C013002088
:10291800F4010020E0140020D8140020AC1400209A
:10292800DC1400200808002000150020FC140020FA
:042938000C1500205A
:10293C0070B5324B1B68002B27D1314B1B681C78B0
:10294C0023005C3B022B16D97D20FDF759FC20207F
:10295C00FDF756FCFFF712FA25006D3D072D15D932
:10296C00713C012C1CD9032D0FD8264B1B681888E1
:10297C0004F069FB09E0244B186801300005000DD8
:10298C0004F061FB2920FDF73BFC70BD2020FDF716
:10299C0037FC5220FDF734FC3A20FDF731FCDFE721
:1029AC00184B1A68194BD31A082BEED90C3A10880D
:1029BC0004F049FB2020FDF723FC2020FDF720FC30
:1029CC00104C2368083B188804F03DFB2020FDF7D1
:1029DC0017FC6920FDF714FC2368043B188804F0ED
:1029EC0032FB2020FDF70CFC7820FDF709FC236856
:1029FC001888013004F027FBC7E7C046F01400200C
:102A0C00E8140020C8140020EC140020C01300208F
:102A1C00204B186800281BD11F4B1B68002B0BD0B8
:102A2C001E4B1B681E4A1268934205D0D01A934263
:102A3C000DD3981AC4300AE01A4B1B681A4A126854
:102A4C00934204D0D01A934201D3981AC4307047E1
:102A5C000238022398430CD00F4B18680028F6D08C
:102A6C000E4B18680E4B1B68984211D00DD2181AD9
:102A7C00EDE70C4B1B680C4A12689342E7D0D01A56
:102A8C009342E4D3981AC430E1E7C01AC430DEE7AD
:102A9C000020DCE764150020881400202415002099
:0C2AAC00281500205415002058150020AB
:102AB80010B5094B1C68221D1A60084B1B68002BB7
:102AC80006D0074B1B78002B02D0064B186801E094
:102AD800FFF7A0FF606010BDC0140020F4010020C3
:082AE8009F150020A814002036
:102AF00010B50B4B1C6800230A4909190A48CA5C27
:102B0000222A03D01A5401334E2BF8D1064A22212F
:102B1000D15401330021D154E318044A136010BD8D
:102B2000941400200C130020701300209C1400202B
:102B30001A4B1B185A781300613B192B03D8203A03
:102B40001300373B05E02F2A1BD91300303B092B1C
:102B5000F6D80F2B18D8114A101882781100613955
:102B6000192907D8203A373A11000F2912D818012D
:102B7000401870472F2A0AD9110030390929F4D991
:102B8000F1E701204042F4E701204042F1E7012053
:102B90004042EEE701204042EBE7C04670130020C0
:102BA000F0B5C64600B50700404B1B680133404AEC
:102BB0001360FFF79DFF002600243E4A03E0013624
:102BC0000134502C10D0A35C5C2BF8D0222BF7D111
:102BD000384B00221A55384B1D68002D0CD1354C4E
:102BE000364B98461E003BE0354A022311680B43E2
:102BF000136080BCB846F0BD012F0ED06320FFF7F4
:102C0000D5FC304A13687600A41B2F49CC540133FD
:102C100013600024274D2E0009E06220FFF7C6FC58
:102C2000EFE7FFF7C3FC0134335D002BE1D0285DF3
:102C30005C28F6D12000FFF77BFF431C03D0033450
:102C4000FFF7B4FCF0E71E4A022311680B43136040
:102C5000CFE7FDF7DBFA0135164B5B5D002BC8D0E3
:102C6000605D5C2807D0012FF3D03368002BF2D0D1
:102C7000FDF7C0FAEFE72800FFF75AFF431C0AD020
:102C80000335012F0DD043461B68002BE4D0C0B2A2
:102C9000FDF7B0FAE0E70A4A022311680B4313601C
:102CA000A7E7C0B2FDF7B2FAD6E7C0469C140020F1
:102CB0009414002070130020F414002064150020E8
:0C2CC000F0140020001500200802002085
:102CCC0010B50F4B1B68032B04D00D4B1B68042B4A
:102CDC0009D010BDFEF7CEF80028F6D0FF2318401F
:102CEC00FEF716F9F1E7074B1B68002BF1D002F049
:102CFC00F3FE0028EDD0FF231840FEF709F9E8E7B2
:082D0C0064150020881400206A
:102D140010B5304B1B68012B0BD0022B1ED0032B9C
:102D240039D0042B33D02C4A402311680B43136051
:102D340010BD2A4B19680A1D1A60294B1B68294AC1
:102D44001268934203D005D2D31A4B60F0E70023F4
:102D54004B60EDE79B1AC4334B60E9E7224B1B68D9
:102D6400002BE0D01D4B19680A1D1A601F4B1B680D
:102D74001F4A1268934203D005D2D31A4B60D7E797
:102D840000234B60D4E79B1AC4334B60D0E7164B47
:102D94001B68002BC7D0FFF797FFFFF795FFFFF7DE
:102DA40093FF0E4B1A68111D1960124B1968124BD0
:102DB4001B68994203D005D25B1A5360B8E700231D
:102DC4005360B5E7094B1968094B1B685B1A20333C
:102DD4005360ADE764150020F0140020C0140020F7
:102DE40054150020581500208814002024150020B4
:0C2DF40028150020741500207815002020
:102E000010B5044B1B68022B00D810BDFFF75EFF06
:082E1000FBE7C0466415002039
:102E180010B50023064A1360064A1360064A136079
:102E2800FFF7EAFFFFF712F90028F9D010BDC046F6
:0C2E38009C140020A0140020F8140020BE
:102E440010B5FFF7DBFF154B1B68022B17D0144B93
:102E54001868002817D0134B1B780020002B12D0C1
:102E6400FFF7DAFD00280ED0FFF7F2F801280BD0A7
:102E740002280CD00C4B1868431E984103E0074B02
:102E840000221A60012010BDFFF7DAFBF2E7064AC0
:102E940080235B0011680B431360EBE7A41400204C
:0C2EA400F40100209F150020F014002015
:102EB00010B5264B1B68012B0BD0022B1AD0032B0D
:102EC00031D0042B2BD0224A402311680B431360CE
:102ED00010BDFDF7D5FF002804D1FFF7B3FF002890
:102EE000F7D0F5E71B4B1A68111D1960FF23184036
:102EF0005060EDE7184B1B68002BE4D002F0F2FDA8
:102F0000002804D1FFF79EFF0028F7D0E0E7114B1F
:102F10001A68111D1960FF2318405060D8E70E4B46
:102F20001B68002BCFD0FEF7A1F8002806D1FFF7D1
:102F3000CDFEFFF787FF0028F5D0C9E7054A1368E3
:102F4000191D11600002000A5860C1E764150020D5
:0C2F5000F0140020C014002088140020A1
:102F5C0010B5094A1368094918680860043B1360E6
:102F6C000C002368002B05D0FDF7F0FAFFF764FF87
:102F7C000028F6D010BDC046C0140020E414002078
:102F8C0010B5044B1A68642311684B431360FFF7A8
:082F9C00DFFF10BDC01400208E
:102FA400114A13681868043B136018280BD90300EE
:102FB400A03B182B05D90D4A8023DB0011680B4375
:102FC40013601F2318400300083B042B04D9042377
:102FD40002009A43122A05D1044A8023DB001168B7
:102FE4000B4313607047C046C0140020F014002047
:102FF40070B5FFF7D5FF174B1B68002B14D10F28B2
:1030040013D844000322A2409023DB05D9689143DE
:10301400D9601968914319601D6801221100A1400B
:103024002943196082409A6170BD44000322A24082
:10303400094BD9689143D9601968914319601D6897
:1030440001221100A14029431960103882409A617D
:0C305400EAE7C046F01400200004004829
:1030600070B5FFF79FFF174B1B68002B15D10F287A
:1030700014D844000322A2409023DB05D968914371
:10308000D9601968914319601D6801221100A1409F
:1030900029431960103082409A6170BD44000322B8
:1030A000A240094BD9689143D960196891431960CE
:1030B0001D6801221100A1402943196082409A61D4
:0C30C000EBE7C046F014002000040048BC
:1030CC0010B5FFF769FF144B1B68002B11D10F28AB
:1030DC0010D84000032282409023DB0519689143ED
:1030EC001960D9689143D960D968012282400A439A
:1030FC00DA6010BD1038400003228240074B19687B
:10310C0091431960D9689143D960D96801228240F2
:10311C000A43DA60EDE7C046F014002000040048D2
:10312C0010B5FFF739FF134B1B68002B11D10F287B
:10313C0010D84000032282409023DB05196891438C
:10314C001960D9689143D960D968022282400A4338
:10315C00DA6010BD400003228240074B196891438E
:10316C001960D9689143D960D968022282400A4318
:0C317C00DA60EEE7F014002000040048C8
:1031880010B5FFF70BFF0E4B1B68002B0CD10F2857
:103198000BD84000032282409023DB051968914335
:1031A8001960D9689143D96010BD4000032282405C
:1031B800044B196891431960D9689143D960F3E7C2
:0831C800F0140020000400488F
:1031D00010B5FFF7E7FE104B1B68002B0FD10F282F
:1031E0000ED89023DB051B8A0122824013400B4935
:1031F0000A68101D0860002B0AD00123536010BD1F
:10320000074B1B8A0F2210400E3A82401340EEE714
:1032100000235360F3E7C046F0140020C0140020E0
:04322000000400485E
:1032240010B5144BDA6814490A40DA6099698022AF
:1032340092000A439A61FCF74DFFFCF74BFFFCF741
:1032440049FFFCF747FF0D4B802212061A6100224A
:10325400DA600B490A6004325A619A6801210A4310
:103264009A60190001220B681A42FCD0FCF732FF65
:1032740010BDC04600100240FFFDFFFF00240140C6
:0432840008270140D6
:103288000C4B1A6801210A431A609A6801310A43F3
:103298009A60190001228B681A42FCD1064B9A6980
:1032A80006490A409A61D968802292000A43DA6086
:1032B8007047C0460024014000100240FFFDFFFF98
:1032C800F0B589B004AA4F4B13CB13C21B881380E7
:1032D8006A464D4B13CB13C21B7813704B4B1B68BC
:1032E8001C68621C18D0072C03D92300A03B072BAD
:1032F8001BD8474B9B699B051ED5464B464A1A600F
:103308000F232340590003228A40072B00D971E07C
:103318009900424841588F46043B3C4A1360FFF7E6
:10332800AFFF684603F001FC35E03D4A8023DB002F
:1033380011680B4313602EE0FFF770FF04A803F039
:10334800F4FBDAE79021C905086810430860C868EB
:103358009043C86001229A4013002E4A93620426C3
:10336800002714000425A3682B43A36023681D428B
:10337800FCD0236CFF18FCF7ABFE013E002EF2D107
:10338800224B1B68BA081A60BB0704D51F4B1A6882
:1033980013680133136009B0F0BD9021C9050868AE
:1033A80010430860C8689043C860D3E79021C905F6
:1033B800086810430860C8689043C860CAE790214D
:1033C800C905086810430860C8689043C860C1E729
:1033D8009021C905086810430860C8689043C86010
:1033E800B8E79021C905086810430860C868904389
:1033F800C860AFE70A4A8023DB0011680B431360FB
:10340800C9E7C046B46E0008C46E0008C0140020A6
:103418000010024000240140FF0700003463000848
:04342800F01400207C
:10342C0010B5074A1368191D1160064A12685A60D4
:10343C00FF20FFF7B5F8FF20FFF7B2F810BDC0462C
:08344C00C0140020001500204F
:10345400F8B5104E33681D6801350F4C2D19280A34
:10346400FF273840FFF7A0F838002840FFF79CF802
:103474000A4B1B68013B1B193268190A1068215456
:103484001268A41863707320FFF78EF83368043B46
:103494003360F8BDC014002008020020001500208D
:1034A40070B57C280DD8C0000E4D441908352D1870
:1034B4002078002804D0FCF7A7FE0134AC42F7D1F1
:1034C40070BD7F2528400001074D441908352D188B
:1034D40020780028F4D0FCF797FE0134AC42F7D1F1
:0C34E400EEE7C04614660008080800204F
:1034F00070B50001064D441908352D1820780028B4
:1035000004D0FCF783FE0134AC42F7D170BDC04655
:043510000808002087
:10351400F0B5C64600B582B0A34B1A6800929B88EA
:103524006A469380A14B1D68002D03D002B080BC75
:10353400B846F0BD9E4B1B689E4A13601B789846A4
:103544001F009D4B1B685E00F6180D20FCF75CFE07
:10355400002E06D02C002020FCF756FE0134A64293
:10356400F9D1944B188803F072FD2020FCF74CFE2F
:10357400404603F06CFD2020FCF746FE7D2F1AD850
:103584004046FFF78DFF682F53D0692F57D06A2F1D
:1035940000D182E06B2F00D187E06C2F56D06E2FC4
:1035A40000D18AE06F2F00D18DE0022342469A4376
:1035B400702A4BD059E02D20FCF726FE3E20FCF764
:1035C40023FE2020FCF720FE4046FFF769FF784BDE
:1035D4001B685B787F241C40662F00D19EE0672F18
:1035E40000D1A5E0612F00D1B7E0744C032D00D1C8
:1035F400C7E02368022B00D8C3E0FCF7ABFFFFF75A
:103604000BFA0028F2D0FEF723FD0500012800D1B3
:10361400ADE0022800D1ADE00428E7D1664B1B6879
:10362400002B00D1ADE0664A1360644B02221A609D
:10363400DCE7644B1B681B68002B07D0C7E7614BB2
:103644001B68191F1A680B689A42C0D0684603F0B9
:103654006EFA574B1B68587800029B781843013068
:1036640003F0F5FC2920FCF7CFFD652F35D1504B35
:103674001B685C782820FCF7C7FD534B1B68102B94
:1036840027D02000FDF706FA2920FCF7BDFD484BA2
:103694001B685B787F241C40A1E74A4B1B681A1FF8
:1036A40012681B689A42D1D291E7464B1B681A1FD5
:1036B40012681B689A42C9D989E7424B1B681B6888
:1036C400002BC3D083E73F4B1B681B68002BBDD185
:1036D4007DE7200003F0BBFCD6E7642F00D076E73B
:1036E400334B1A6893781B04517809060B431179FC
:1036F4000B43D47824021C432820FCF785FD324B6D
:103704001B68102B06D02000FDF7C4F92920FCF714
:103714007BFD67E7200003F09AFCF7E72820FCF71D
:1037240073FD2000FFF7E2FE2920FCF76DFD5CE746
:103734002820FCF769FD2000FFF7D8FE4020FCF7A5
:1037440063FD20010830214C00190004000C03F033
:10375400B4FC2920FCF758FD47E72020FCF754FD72
:103764003C20FCF751FD2D20FCF74EFD3DE7FEF714
:1037740067FF3BE70D4A80235B0011680B4313602E
:10378400D4E62020FCF740FD43465C3B022B03D8E3
:10379400684603F0CCF9C9E67B20FCF735FD202010
:1037A400FCF732FDC2E6C046906B0008F01400201E
:1037B400EC140020E8140020E0140020F4010020A0
:1037C4000C150020C0140020AC14002008080020B0
:1037D40010B5FFF79DFE074B1B68002B08D1064B65
:1037E4001B681B789B00054A9B589847FFF7A4F871
:1037F40010BDC046F0140020EC140020000000208E
:1038040010B51B4A1368013313601A4B1A68111D53
:10381400196019490B6853601A787F2313401B0100
:10382400164AD3189B680B601B787C2B0BD8144A60
:103834001268032A04D09B00124A9B58984710BD73
:10384400FFF7C6FFFBE70E4B1B68032B06D00E4B9E
:103854001B68002BF3D1FFF7D3FFF0E7FFF758FE07
:10386400094B1B68002BEAD1FFF766F8EFE7C04667
:10387400E0140020C8140020EC14002008080020E4
:0C388400F401002000000020F0140020DF
:10389000F0B587B001AA3D4B13CB13C211001A68D3
:1038A0000A601B790B713A4C3A4BE4183A4B1B688F
:1038B000A34265D2394D384E2F003DE0FEF7BCF9EA
:1038C00041E0FFF79FFF28E0FFF7A8F800280CD1A0
:1038D00033681B787C2B1BD8304A1268032A14D01B
:1038E0009B002F4A9B58984717E0FEF7B3FB01282F
:1038F00008D00228ECD12B4A80235B0011680B43CF
:1039000013603DE0FEF79EFEE2E7FFF763FF04E091
:103910003B68032B21D0FFF775FFFFF771FA214BAE
:103920001B68002B2CD11C4B1B68002B1AD00133B9
:10393000194A1360A34223D22B68002BC4D11A4B1F
:103940001B68042BBAD0144B1B681B787C2BB8D88F
:103950009B00134A9B589847DFE7FFF7DBFDFEF714
:10396000EDFFD8E70D4B1B68032B0BD00B4B01224F
:103970001A6000230D4A13700D4A13600D4A13603C
:1039800007B0F0BD01A803F0D4F8EFE7DC6E000843
:1039900008020020F80D0020EC140020F4010020A3
:1039A00000000020F0140020A41400209F15002027
:0839B00008150020E0140020BE
:1039B800F8B5274B1C68002C2ED1264B1B68190123
:1039C800254A5218D168C022120511420AD0234A4A
:1039D8001168081D10601B011F4AD3189B684B60B3
:1039E8002000F8BD1B011C4AD3189A681C4B1A60AA
:1039F8001C4B01221A701C4D2F681C4C2668522340
:103A08002B6023601A4B00221A60FFF73DFF2F60DE
:103A18002660184B1C68E3E70E4B186802010E4B32
:103A28009B18DA68C0231B0514001C401A4204D1F5
:103A380080231843FEF7B6FDD2E76620FEF7B2FDF5
:103A4800044B1868FEF7AEFD0A4B1C68C8E7C04671
:103A5800F4140020CC14002008080020C014002012
:103A6800EC1400209F150020A01400209C140020B6
:083A7800F8140020F0140020F6
:103A800070B50023384A1370384A1360384A1360FF
:103A90001500384E0EE0384B1B68FF2B24D86520EC
:103AA000FEF784FD344B1868FEF780FD304B1A6832
:103AB0002E4B1A60314C2B682268934230D2FEF7AD
:103AC000C1FB3378002BF6D0FEF75CFC00281FD03A
:103AD0002B4B1B68002BDED12A4A1368191D11607D
:103AE000254A12685A60E1E76420FEF75FFD224C28
:103AF00003202056FEF75AFD0223E05EFEF756FD36
:103B000023681812FEF752FD2068FEF74FFDCDE73F
:103B1000FEF7E2FC002809D0FFF74EFF002800D096
:103B200070BD134B1A68114B1A60C3E7FEF798FC7F
:103B300000280AD0FEF752FD134B1B68002BEFD173
:103B40000B4B1A68094B1A60B4E70F4A012311683E
:103B50000B4313600D4B1A680D4B1A60044B1A6827
:103B6000024B1A60DCE7C0469F1500209414002029
:103B70009C1400207013002098140020A014002032
:103B8000F4140020C0140020F0140020FC140020C5
:043B900000150020FC
:103B9400F0B5DE4657464E464546E0B591B00BA912
:103BA400B94B0A0013CB13C203CB03C206AAB74B0B
:103BB40013CB13C211001A680A609A888A809B7911
:103BC4008B7102AAB24B13CB13C21B881380B14B67
:103BD4001A68B14B1A60FEF733FBFEF77BFC002832
:103BE4000DD1FEF73BFC002805D1AC4A0123116836
:103BF4000B43136018E10BA802F099FF14E1A54BE5
:103C04001A68A54B1A6006A802F091FFA44D2B6810
:103C14001801A44C001903F050FA0D20FCF7F4FA33
:103C24002B681A01A418E168C0221205080010408C
:103C34000190114200D0FEE01B019A4AD3189C68FF
:103C4400994BE41A2405240D1B5D0125612B00D139
:103C5400D1E0954E24E00D20FCF7D6FA019D1FE03B
:103C6400914B1A195078000202341F5D0743282033
:103C7400FCF7CAFA781C03F0EAF92920FCF7C4FA25
:103C840001352020FCF7C0FA2020FCF7BDFA0134EE
:103C9400854B1B5D612B00D1ADE00135072DDAD8D2
:103CA400A0190004000C03F0D2F93A20FCF7ACFA96
:103CB400305DFFF7F5FB335D1A00683A0A2ACFD965
:103CC400652B1AD0642B2ED0662B4CD0672B57D083
:103CD400622BD6D12220FCF797FA734B1B195B7821
:103CE4009B46A31C98465B46002B7DD06E4B4344F9
:103CF40099465C460F239A466BE001342820FCF772
:103D040083FA6A4B1B68102B08D0674B185DFCF7CD
:103D1400C1FE2920FCF778FA0135B2E7624B185D41
:103D240003F0CBF9F5E76048021993781B04517846
:103D340009060B43D7783F020434025D13431F4343
:103D44002820FCF761FA594B1B68102B07D0380068
:103D5400FCF7A0FE2920FCF757FA013591E738005B
:103D640003F0ABF9F6E701342820FCF74DFA4E4B8B
:103D7400185DFFF7BBFB2920FCF746FA013580E705
:103D840001342820FCF740FA474B1F5D3800FFF749
:103D9400ADFB3F01083743483F184020FCF734FA95
:103DA4003804000C03F089F92920FCF72DFA0135B9
:103DB40067E75C20FCF728FA3809FCF71BFB504640
:103DC4003840FCF717FB013C01239C46E144002CDE
:103DD40009D04B461F783B00203B5E2BE9D83800C6
:103DE400FCF712FAEFE7D8444446013C2220FCF7E2
:103DF4000BFA033545E72C4820180004000C03F0A7
:103E040026F93A20FCF700FA3B20FCF7FDF9244B95
:103E14001A681201234B9B18DA68C0231B051A4247
:103E240009D10D20FCF7F0F911B0F0BCBB46B24645
:103E3400A946A046F0BD02A802F079FE1B4B1B6800
:103E4400102B18D0164B1A681201164B9B18986841
:103E540002F09FFE2020FCF7D7F94020FCF7D4F9AC
:103E64000F4B1868000108300E4BC0180004000CFA
:103E740003F023F9D5E70A4B1A681201094B9B1882
:103E8400986803F01AF9E5E7A46B0008B86B00081A
:103E9400CC6B00089C14002094140020F014002023
:103EA400CC1400200808002008020020AC140020D4
:103EB400134B1B68134A1360134A12681201134907
:103EC4005218BE20C000844661448A420AD2104976
:103ED4000139891A8908013189005118002001C269
:103EE4008A42FCD10B4A934209D80B4A9B180B49CE
:103EF4008C4662440021197001339342FBD1704710
:103F040000150020FC140020DC1400200808002008
:103F1400F80D0020FE05000008020020FF05000047
:103F240010B5164B1A68164B1A60FEF789F9FEF79E
:103F3400D1FA00280DD0114B1A68114B1A60114B9D
:103F44001B68032B0BD8104A802311680B431360A2
:103F540004E00D4A212311680B43136010BD0B4A82
:103F640013600B4A1B0100219954D318DB681B050D
:103F74001B0D084A1360FFF79BFFEFE79C1400201A
:103F840094140020CC140020F0140020DC14002031
:083F94000808002000150020C0
:103F9C0010B50023204A1360204A1360204A137086
:103FAC00204A1360204A1360204A01211160204AE4
:103FBC001360204B1A68204B1A60204A002311789A
:103FCC00002903D0013310325F2BF8D11C4A136047
:103FDC001C4A1D4BD35C612B1CD01B4B1100013BAD
:103FEC00CA5C612A02D0002BF9D102E0002B00D070
:103FFC000133164A1360FFF757FF154A154B1A6029
:10400C0000231360144A0F491160144A1360FDF722
:10401C0065FC10BD0C4BEBE7F8140020F4140020E9
:10402C009F15002008150020E0140020F40100204A
:10403C00A8140020D8140020AC140020080800207C
:10404C00DC14002008020020FF05000000150020F1
:10405C00C0130020C8140020EC140020F014002021
:10406C0030B5B9B036AAA04B1968369199889180B1
:10407C009B79937134AA9D4B1968349199889180DE
:10408C009B79937131AA9A4B03CB03C211001A8806
:10409C000A809B788B702EAA964B13CB13C22BAA3B
:1040AC00954B03CB03C211001A880A809B788B7046
:1040BC0027AA924B13CB13C21B88138022A9904BB7
:1040CC000A0013CB13C203CB03C21CA98D4B0A00ED
:1040DC0013CB13C203CB03C21B78137018AA8A4BE1
:1040EC0013CB13C21B68136014AA884B13CB13C2D7
:1040FC001B8813800FAA864B13CB13C211001A68AE
:10410C000A609B888B8009A9824B0A0013CB13C2CF
:10411C0003CB03C21B78137005AA7F4B13CB13C2BE
:10412C001B78137001AA7D4B13CB13C21B88138011
:10413C007B4B1A687B4B40339A4200D280E07A4921
:10414C000423086803430B60764B0C339A4204D269
:10415C00754A042311680B431360744B1B68002BC6
:10416C000FD0734B1968734B09010022CA545B18AA
:10417C005A709A70DA701A715A719A71DA719A606F
:10418C00DA606A4B00221A606B4B1B68002B0ED056
:10419C000024694D2020FCF733F801342B68A3422E
:1041AC00F8D85E20FCF72CF80D20FCF729F836A87F
:1041BC0002F0B9FC5C4C206802F045FF3D20FCF796
:1041CC001FF82368DB075ED4574B1B689B075ED434
:1041DC00554B1B685B075ED4534B1B681B075ED4A7
:1041EC00514B1B685B065ED44F4B1B689B065ED421
:1041FC004D4B1B681B065ED44B4B1B68DB055ED41A
:10420C00494B1B689B055ED4474B1B685B055ED412
:10421C00454B1B681B055ED434A802F084FC464B4E
:10422C001868FCF733FC2920FBF7EAFFFFF7B0FE18
:10423C000D20FBF7E5FF414B00221A6039B030BD71
:10424C00384B0C339A4200D282E7374B1B68002B59
:10425C0000D082E7354B1B68002B40D1384B1B68D4
:10426C00012BE5D02020FBF7CBFF6F20FBF7C8FF1D
:10427C006B20FBF7C5FF334B1B68102BD8D14820A4
:10428C00FBF7BEFFD4E731A802F04DFC9CE72EA84B
:10429C0002F049FC9CE72BA802F045FC9CE727A800
:1042AC0002F041FC9CE722A802F03DFC9CE71CA814
:1042BC0002F039FC9CE718A802F035FC9CE70FA82B
:1042CC0002F031FC9CE714A802F02DFC9CE709A835
:1042DC0002F029FC9CE705A802F025FC9CE701A84C
:1042EC0002F021FCA4E7C046106C0008186C000812
:1042FC00206C00082C6C0008386C0008446C00081A
:10430C00546C0008686C0008806C0008906C000805
:10431C00A06C0008B46C0008CC6C0008DC6C0008C5
:10432C00C014002010140020F0140020F4140020FD
:10433C00DC1400200808002094140020081500202C
:08434C00F8140020AC1400205D
:1043540010B50023134A13600A2213490A60134953
:104364000A60134A01211160124A1360124B312270
:1043740056240021C02000051C705A709970D86022
:10438400996010330132D2B2352AF5D10B4B313A50
:104394001A60002308493C328B54094A1360FFF722
:1043A400FBFD10BD6C150020D8140020AC140020B7
:1043B400F40100201015002008080020DC1400205F
:0443C40000150020C0
:1043C80070B5164C164D2B682360FDF737FF2B6828
:1043D8002360144B1D68013D28006B1C17D02D016C
:1043E800114BED18114E10E08B420BD1002913D060
:1043F8000132A95C935D1C00613C192CF4D8203B68
:10440800DBB2F1E7103D013804D30022F1E70120C7
:10441800404201E00120404270BDC0469414002093
:104428009C140020DC1400200808002070130020D1
:1044380010B5FFF7C5FF0400431C0DD002011D4B4A
:104448009B18DA68C0231B051A420BD01A4A80232E
:1044580011680B43136010BD174A212311680B43E1
:104468001360F8E7FFF7ACFF431C11D00201114BB2
:104478009B18DA68C0231B051A420FD1844213D94E
:104488000C4B24011C19A268000118188260E2E78D
:10449800094A212311680B431360DCE7064A80238D
:1044A80011680B431360D6E7034A802311680B4356
:0C44B8001360D0E708080020F01400207A
:1044C40010B5FFF77FFF431C0FD003010D4AD2182C
:1044D400D3681B051B0D0C495B1892689A420AD3DA
:1044E4000001084A1018836010BD084A212311688E
:1044F4000B431360F8E7054A802311680B431360EC
:10450400F2E7C0460808002008020020F01400204A
:10451400F8B506000D490A68571C0F6054783F1916
:10452400002C10D00D0005E05878FBF76DFE013C1F
:10453400002C08D02B685A1C2A60012EF4D058781D
:10454400FBF72EFFF3E7014B1F60F8BDEC140020CE
:10455400074B1A68511C196051780902901C1860A5
:1045640092781143802292050A431A607047C0462C
:04457400EC14002023
:1045780010B5084B1B681B68002B08D0064A136847
:1045880002331360034A1368043B136010BDFFF73E
:0C459800DDFFF7E7C0140020EC14002049
:1045A40010B5094B1B68191F1A680B689A4208D189
:1045B400064A136802331360034A1368043B13600A
:1045C40010BDFFF7C5FFF7E7C0140020EC1400206E
:1045D40010B5094B1B68191F1A680B689A4208DD4D
:1045E400064A136802331360034A1368043B1360DA
:1045F40010BDFFF7ADFFF7E7C0140020EC14002056
:1046040010B5094B1B68191F1A680B689A4208DA1F
:10461400064A136802331360034A1368043B1360A9
:1046240010BDFFF795FFF7E7C0140020EC1400203D
:1046340010B584B001A8214B020012CB12C21B8812
:10464400138002F074FA1E4C2068FCF723FA2368E6
:104654001F2B15D00B2B1DD0194B1B68132B20D0EF
:10466400174B1B68262B20D0154B1B68392B20D0E9
:104674003020FBF7C9FD3020FBF7C6FD04B010BDA8
:104684003220FBF7C1FD3520FBF7BEFD3020FBF7E0
:10469400BBFDF3E73520FBF7B7FD3220FBF7B4FD94
:1046A400DAE73220FBF7B0FDDAE73420FBF7ACFDA4
:1046B400DAE73620FBF7A8FDDAE7C046F46C000819
:0446C4008815002035
:1046C80070B59CB0674B1A681A929A8869466C2034
:1046D80009180A809B796A466E215218137018AD22
:1046E800614B2A0003CB03C2604B1A6816929A8862
:1046F80069465C2009180A809B796A465E2152182F
:10470800137012AC5A4B220043CB43C21B78137070
:10471800584B1A6810929A8810AB9A80564B1A68B0
:104728000E929A880EAB9A800AAA544B43CB43C286
:104738001B68136007AA524B43CB43C203AA514BD1
:1047480043CB43C21B6813606A464F4B03CB03C27B
:104758001B8813804420FBF755FD6120FBF752FDB1
:104768007420FBF74FFD6120FBF74CFD1AA802F0FF
:10477800DCF946480C3002F068FC280002F0D5F954
:104788001AA802F0D2F9424802F05FFC200002F0B9
:10479800CCF9404802F059FC16A802F0C6F93E4888
:1047A80002F053FC0D20FBF72DFD3C4B1B68002B42
:1047B80010D110A802F0B9F90AA802F0B6F907A8B2
:1047C80002F0B3F9364B1B680024002B06D0324E9A
:1047D800334D3BE00EA802F0A8F9EDE76E20FBF799
:1047E80011FD6F20FBF70EFD6E20FBF70BFD65201A
:1047F800FBF708FD0D20FBF705FD03A802F095F96E
:10480800284B18683030C0B2FBF7FCFC2020FBF7BF
:10481800F9FC2020FBF7F6FCFFF708FF684602F0DA
:1048280084F9214B1868002818D16130FBF7EAFC9D
:104838006C20FBF7E7FC6C20FBF7E4FC0D20FBF792
:10484800E1FC1CB070BDFBF7DDFC01342B68013BBB
:104858001B01F318185D0028F5D1CBE7FCF718F910
:10486800ECE7C046086D0008106D0008186D0008D8
:10487800206D0008306D0008386D0008406D000894
:10488800506D00085C6D00086C6D00081014002065
:10489800C013002008020020080800206C15002022
:0C48A8001015002064150020841500206D
:1048B40030B58BB003A8124B020032CB32C232CBDC
:1048C40032C21B8813806A460E4B32CB32C202F0CE
:1048D4002EF9FCF7FFFA0028FBD0FF2318405928D3
:1048E40008D0684602F023F90D20FBF78DFC002068
:1048F4000BB030BD0D20FBF787FC0120F8E7C04664
:08490400546300087063000811
:10490C00F0B591B0040001A9334B0A0023CB23C2AC
:10491C0023CB23C223CB23C203CB03C22F4D304E58
:10492C0033682B60FDF788FC33682B60FDF724FDA2
:10493C00051E08D02B4A802311680B4313600025F9
:10494C00280011B0F0BDFDF785FD002804D10CA89E
:10495C0001002A00244F0EE001A802F0E4F8FFF752
:10496C00A3FF0028F3D10225EAE7002B12D0072A77
:10497C000AD001320131D35D0B701E00613E192E3D
:10498C00F3D8203B0B70F2E7164A022311680B4355
:10499C001360D5E70CAB1B78002B0CD0134A1268B4
:1049AC00120113495218535501354378002B02D08C
:1049BC000130072DF7D10D4B1A6812010C4B9B18C7
:1049CC005D1900226A700B4A10680B4A82189A60B3
:1049DC002043D8600125B3E77C63000894140020C1
:1049EC009C140020F014002070130020DC14002014
:0C49FC0008080020001500200802002020
:104A080070B5C0200005FFF77DFF00280DD00A4CC7
:104A180022680A4803681D010949491915688D600B
:104A2800043A22600133036070BD064A012311680D
:104A38000B431360F8E7C046C0140020DC140020C4
:084A480008080020F014002012
:104A500010B50020FFF75AFF002808D0022807D021
:104A6000074B1A68074B1A60074B01221A6010BDEA
:104A7000064B1B681B01064A00219954F7E7C04604
:104A800000150020FC140020F4140020DC14002089
:044A900008080020F2
:104A940010B590B008A9284B0A0013CB13C213CB4E
:104AA40013C203CB03C201A9244B0A0013CB13C2C4
:104AB40013CB13C21B681360214A13681C68043BA0
:104AC4001360962C1ED0112C29D0192C03D1132439
:104AD4000B2C1BD002E0312C15D11F24132C15D024
:104AE4001F2C13D0262C11D0392C0FD0602C0DD0B4
:104AF40001A802F01CF8134A8023DB0011680B4361
:104B040013600AE06024382C0AD1262408A802F095
:104B14000EF8FFF7CDFE002806D110B010BD0B240F
:104B2400572CD5D13924F1E7074B1C60074B1C6087
:104B3400FBF7DCFAF1E7C046A8630008C863000885
:104B4400C0140020F0140020881500205C150020FB
:104B540010B592B00AA93A4B0A0013CB13C213CB77
:104B640013C203CB03C201A9364B0A0013CB13C2F1
:104B740013CB13C203CB03C21B881380324A1368BE
:104B84001C68191F1160314A1268A24220D0304AB1
:104B94001268002A14D0043B1B68042B1AD8A31EE5
:104BA400022293431DD0012C26D0032C34D0294B50
:104BB4001B68294A12689A4229D1244B1C6007E0D9
:104BC400264A802311680B431360204B00221A608D
:104BD40012B010BD214A8023DB0011680B4313601F
:104BE400F6E70AA801F0A3FF0D20FBF70DFBFFF782
:104BF4005FFE0028D7D1EBE701A801F098FF0D2054
:104C0400FBF702FBFFF754FE0028D0D1E0E7124A7D
:104C14001360FBF76BFAD0E701A801F088FF0D20C1
:104C2400FBF7F2FAFFF744FE0028D1D00A4B094AF9
:104C3400196811601F221A60FBF758FABDE7C046D5
:104C4400846D0008A46D0008C014002064150020C1
:104C5400881400205C15002088150020F014002022
:104C640030B585B0174B1A6802929A8869468A81D2
:104C74009B798B73144B1A6800929A888A809B796B
:104C84008B71FCF7C5FA114C23681D6802A801F06A
:104C94004EFFFDF767F82020FBF7B6FA23681C687F
:104CA400684601F044FFFDF75DF82020FBF7ACFAFD
:104CB400FFF7FEFD002803D0054B1D60054B1C606B
:104CC40005B030BD906F0008986F0008C014002034
:084CD4001415002070150020EA
:104CDC0030B589B001A80B4B020032CB32C232CBBB
:104CEC0032C21B68136001F01EFFFFF7DDFD0028C8
:104CFC0001D109B030BDFBF7B5FC034B01221A60A2
:0C4D0C00F7E7C046E46300086C150020C7
:104D180010B58CB006A91E4B0A0013CB13C203CBE7
:104D280003C21B78137069461A4B0A0013CB13C2CF
:104D380003CB03C21B781370174A13681968043B26
:104D4800136001290ED8002914D1684601F0EDFE40
:104D5800FFF7ACFD00280BD0104B00221A60FFF7BC
:104D6800F5FA05E00E4A8023DB0011680B43136057
:104D78000CB010BD06A801F0D8FEFFF797FD00287B
:104D8800F6D0064B01221A600120FBF75DFAEFE727
:104D9800186F0008306F0008C01400206C15002040
:044DA800F0140020E3
:104DAC00074B1B68002B09D0054B00221A60054AE3
:104DBC001368191D1160044A12685A607047C04686
:0C4DCC0008150020C01400200415002071
:104DD80010B5214B1A68214B1A60FDF72FFAFDF721
:104DE80077FB002821D01C4B1A681C4B1A601C4BFF
:104DF8001A6812011B4B9B18DA68C0231B051A425C
:104E080019D0194B1B78002B1BD1184B1B68002B92
:104E18001AD117480368124A11680901114A521831
:104E280019689160043B036004E0124AA0231168EA
:104E38000B43136010BD0F4A802311680B431360A6
:104E4800F8E7FFF7AFFFE0E76720FDF7ABFB044BA0
:104E58001868FDF7A7FBEDE79C14002094140020C8
:104E6800CC140020080800209F150020F41400200E
:084E7800C0140020F01400201A
:104E8000F0B5C64600B588B069462B4B0A0013CB77
:104E900013C213CB13C203CB03C2284B1B78002BC6
:104EA00014D1274A13688024A40519680C43043BD5
:104EB0001360244B9C420CD9234A8023DB001168E9
:104EC0000B43136008B080BCB846F0BDFFF76EFF1F
:104ED000E7E70D20FBF79AF9684601F02AFE20006B
:104EE00002F0B7F8270080370F25032398460FE01C
:104EF0000D20FBF78BF9200002F0ABF83A20FBF70E
:104F000085F9300001F02BFE00250134BC420ED0A3
:104F100026780135102DEBD0300001F020FE4346FD
:104F20002B40032BF1D17C20FBF770F9EDE70D202E
:104F3000FBF76CF9C6E7C046006400089F15002027
:0C4F4000C0140020807F0020F01400202E
:104F4C0082B03A4B1A6801210A431A605A683848F1
:104F5C0002405A601A68374802401A601A6836488C
:104F6C0002401A605A68354802405A60DA6A0F20CB
:104F7C008243DA621A6B324802401A635A6B8A43D4
:104F8C005A6300229A6000920192196880225202A0
:104F9C000A431A60190080229202A020C0010B68FB
:104FAC0013400193009B01330093019B002B02D112
:104FBC00009B8342F3D11D4B1B689B0306D5012339
:104FCC000193019B012B04D002B070470023019385
:104FDC00F7E71C4B11221A60144B5A685A605A6836
:104FEC005A605A6818490A405A6059688822520314
:104FFC000A435A601968802252040A431A60190045
:10500C00802292040B681342FCD0084B5A6803218F
:10501C008A435A605A6801390A435A6019000C22B3
:10502C004B681340082BFBD1CEE7C0460010024062
:10503C000CB8FFF8FFFFF6FEFFFFFBFFFFFFC0FF02
:0C504C00ACFEFFFF00200240FF7FC0FF11
:105058000E4B00221A609022D20513680C490B40AF
:1050680013600C4A802380210906D150BFF34F8F6B
:10507800BFF36F8F084B1969802212040A431A6123
:10508800DA6906490A40DA617047C0468814002088
:10509800FFFF3FFC00E100E000100240FFFF7FFF40
:1050A8004C4B80221A6000224B4B1A604B4908680F
:1050B80080231B0203430B60494B1A601B68494A53
:1050C8009A1849490A6049490A604949581849499A
:1050D80008604949581849490860494958184949D0
:1050E80008604949581849490860494958184949C0
:1050F8000860494958184949086049498C46634439
:1051080048490B60484B1B68002B06D11300183325
:1051180046490B60464902330B6040231380354BE8
:105128001B6800221A80354B1B6880211980354B7B
:105138001B6840491980354B1B6880204000188047
:10514800344B1B681A80284B1B689881DA81013020
:10515800FF3018825A82314B1B681880314B1B680C
:105168001980314B1B68002B0BD1304B1B68C021B9
:10517800890019802E4B1B681A801B4B1B6899836A
:10518800DA832D4B2D4A1A802D4B2E4A1A802E4B2E
:105198002E4A1A80244B1B68002B02D12C4B2D4A17
:1051A8001A802D4BBF2212021A6000232B4A13606B
:1051B8002B4A13602B4A2C490A602C490A602C4A56
:1051C8002C490A602C490A602C4A13702C4A137027
:1051D8007047C0464C5C004090140020585C00406A
:1051E800505C0040006000408C1400204C150020EA
:1051F800026000403815002004600040501500206F
:10520800066000403C15002008600040481500205A
:105218000A60004034150020146000404415002046
:10522800166000403015002084140020401500202E
:105238002C1500200084FFFF005C00402032000095
:10524800045C004031300000085C0040323000004F
:105258000C5C004033360000405C004070140020B5
:1052680088140020F80D0020201500201C150020AF
:10527800C41100202815002024150020F910002052
:04528800921500205B
:10528C0070B5204CE36980252D042B43E361FAF7BC
:10529C001DFF23691D432561FAF718FF236B80223C
:1052AC00134323632369184A134023619022D205C8
:1052BC00136816490B401360154B0021154A1980D1
:1052CC0002339342FBD1144B0021144A1980023350
:1052DC009342FBD1124A116880231B020B431360CB
:1052EC00104C01232360C820FBF7AEF90023236088
:1052FC00094A1360FFF7D2FE0B4B802212061A608C
:10530C0070BDC04600100240FFFF7FFFFFFF3FFC57
:10531C00005C0040205C0040445C0040605C00404D
:0C532C00585C0040405C004000E100E0E4
:1053380070B582B0284B1B68402B45D9274B1B689A
:1053480040221A80244A1368403B1360234B1B6891
:105358001B88002B16D0224C002122481F4D0368C1
:105368001E785A1C02605A780233036013023343D2
:1053780023800234013189B22B681B8801335B100A
:105388009942ECDB184B1B881B0604D5164A138878
:1053980016490B401380164B1B68164A1A80124B8D
:1053A8001B889BB26A46D380D3889B0602D40E4BD7
:1053B800114A1A806B4606331B88DB0602D40A4B57
:1053C8000E4A1A8002B070BD034B1968034A12686E
:1053D800118000221A60B9E77014002038150020E7
:1053E800406000407C140020005C00400F8FFFFFED
:1053F8003C1500200084FFFFA082FFFF9082FFFF82
:1054080082B0174B1B6800221A80164B1B881B069C
:1054180004D5144A138814490B401380104B1B6899
:1054280000221A800F4B1B889BB26A46D380D38810
:105438009B0602D40B4B0D4A1A806B4606331B8819
:10544800DB0602D4074B0A4A1A806B4606331B88D0
:105458005B0402D5034B074A1A8002B07047C04666
:1054680038150020005C00400F8FFFFFA082FFFF6F
:085478009082FFFF80C2FFFFDC
:1054800000B583B01C4A13881C490B4013801C4B89
:105490001B68052B1DD01B4B1B68002B29D1164BFD
:1054A0001B881BB2002B1EDB134B1B889BB26A466A
:1054B000D380D3889B0402D40F4B134A1A806B46C7
:1054C00006331B88DB0402D40B4B104A1A8003B04E
:1054D00000BD0F4B1B68802213430E4A1360084B1C
:1054E00000221A60D7E7044A13880B490B40138047
:1054F000DAE7FFF721FFEAE7005C00400F8FFFFFCC
:10550000741400207014002080A2FFFF8092FFFF1F
:0C551000901400204C5C00408F0F000045
:10551C0082B0134B1A8813490A401A801B881B0649
:10552C0004D50F4A138810490B4013800C4B1B8871
:10553C009BB26A46D380D388DB0602D4084B0B4A55
:10554C001A806B46DA8806331B889B0402D4044B02
:10555C00074A1A806B4606331B8802B07047C04658
:10556C00005C00408F0F00000F8FFFFF9082FFFF49
:04557C0080A2FFFF0B
:1055800030B587B0C54B1B881B0500D4D0E1C34A9A
:105590001388C3490B401380C24B1B78C2490B7060
:1055A000C24B1A78C24B1A70C24B1A88C24B1A806F
:1055B0001A88120AC14802701B88DBB2C04A1370F5
:1055C000C04B1A88C04B1A80C04B1A88C04B1A8037
:1055D000C04B00221A60C04B1B68C04A1A800B786F
:1055E000212B31D0B04B1B78DBB2A12B62D0AE4B5C
:1055F0001A7861231A4206D0AB4B1B786122134004
:10560000012B00D046E1A54A1388A5490B40138021
:10561000A74B1A78D3B2062A00D17DE0062B66D8B4
:10562000002B70D0052B00D025E1AD4B00221A6075
:10563000FFF7EAFEA04B1B887F221340A94A1360A4
:10564000A44B05221A607FE1994B1B78202B0BD0CD
:10565000974B1B78222B2AD1904A138890490B40F4
:105660001380FFF7D1FE6FE18C4B1B889BB2162293
:105670006A44138013889B0402D4884B9A4A1A8088
:1056800016236B441B88DB0402D4844B974A1A8090
:1056900016236B441B885B0403D5804BA022920029
:1056A0001A807E4A13881BB2002BFBDB4CE1FFF70C
:1056B00035FF49E17E4B1B78212B98D1774A13881F
:1056C00077490B401380864A07231360804B1B8861
:1056D0009BB21268934204D27D4B1B889BB2804AD6
:1056E0001360834B834A1A60FFF726FE2CE1092BD7
:1056F00000D0C0E07A4B00221A60FFF785FE7E4B97
:10570000FF221A6020E1764B02221A60784B7B4A16
:105710001A60FFF711FE17E1684B1B78012B28D0A8
:10572000664B1B78022B5ED0644B1B78032B00D09A
:105730009EE0634B1B78012B73D0614B1B78022BCF
:1057400000D180E05E4B1B78002B00D08DE0644AD6
:10575000043313605E4B1B889BB21268934204D2E1
:105760005B4B1B889BB25E4A1360614B644A1A60B4
:1057700028E05B4B12221A60624B1B68012B24D07D
:10578000614D5B4B1D60614B1C68614A0123944273
:105790001DD0681E6A46D11CC25CCA540133132B4B
:1057A000FAD101AB1C72240A5C725A4B9D4215D08F
:1057B000594B1A7801AB9A72574A1268120ADA7278
:1057C0004B4A1360FFF7B8FDBEE0524DD9E7534B8B
:1057D000514A12689A42F5D00123DAE74E4B1A6813
:1057E0000332D2B2E6E7474B1B68012B12D03C4B89
:1057F00043221A603E4B4A4A1A60354B1B889BB2C3
:10580000374A12689342DDD2314B1B889BB2344A2F
:105810001360D7E7324B65221A60354B414A1A6054
:10582000EBE72F4A17331360294B1B889BB2126892
:10583000934204D2264B1B889BB2294A13602C4BFF
:10584000394A1A60BEE7264A10331360204B1B8882
:105850009BB21268934204D21D4B1B889BB2204A14
:105860001360234B314A1A60ACE7FFF757FE6BE039
:10587000FFF754FE68E00C4B1B78002B02D0FFF7BB
:105880004DFE61E0054A138805490B401380FFF780
:10589000BBFD59E0FFF742FE56E0C046005C004009
:1058A0008F0F000080600040931500208160004051
:1058B0009415002082600040FA1000209C15002002
:1058C0009D150020846000409015002086600040F7
:1058D0008A120020741400203C1500200084FFFF71
:1058E000701400209014002080A2FFFF8092FFFF20
:1058F0007C140020E46F000888140020F46D000878
:10590000FC69000884140020D46D000814150020E0
:1059100083040000246E000870150020405700002A
:10592000A06F0008EC6F0008006A0008046E000811
:10593000094B1B889BB216226A44138013881BB242
:10594000002B03DBFFF760FD07B030BD1388034A6F
:105950001340014A1380F5E7005C00408F0F000000
:10596000F0B5DE4657464E464546E0B583B03C4B63
:105970001B881B0604D53A4A13883A490B4013800A
:10598000394C0022394FB846394B9C46BA46B94685
:1059900033E05346374E1E6044E001AB1B882B803A
:1059A0005A46354B1B681A802D4B1B889BB26A46A2
:1059B000D380D3889B0602D4294B304A1A806B4689
:1059C00006331B88DB0602D4254B2D4A1A8003B010
:1059D000F0BCBB46B246A946A046F0BD254B2349C4
:1059E0000B600232D2B26B46598801AB1B880902A8
:1059F0000B432B80402AD4D00234A51E3B6821499A
:105A000008688342CDD0694600264E8019788B46BF
:105A100001A95E460E80013341460B60614609686C
:105A20008B42B6D0531CDBB29B46402BB5D04B46C5
:105A30001B6883420AD01878834668465E464680D3
:105A400001339942CAD009490B60CAE76B465A88AC
:105A500001AB1B88120213432B805A46CCE7C04689
:105A6000045C00400F8FFFFF026100401C15002006
:105A7000F8010020F80D002034150020A180FFFF60
:085A80009180FFFF20150020BA
:105A880082B0114B1B881B0604D50F4A13880F4997
:105A98000B4013800E4B1B6800221A800A4B1B8890
:105AA8009BB26A46D380D3889B0602D4064B094A28
:105AB8001A806B4606331B88DB0602D4024B064A63
:105AC8001A8002B07047C0460C5C00400F8FFFFF81
:0C5AD8002C150020A386FFFF9386FFFF23
:105AE40010B5204B1B68002B34D01F4B18680028BE
:105AF4002FD01E4B1A681E4B1B689A4230D0511C83
:105B04001A48016014781B4A1268914225D0174A3A
:105B14001268991A934201D2C433991A164B1B681E
:105B2400002B11D07D290FD8134B00221A60134B80
:105B34001B889AB29B0402D4104B11491980D304D8
:105B440002D40E4B0F4A1A80FAF7B8FA80200002EA
:105B5400204310BDFAF7FEFCC7E70B490160D6E706
:105B64000020F6E768150020881400202415002082
:105B740028150020FC01002078140020085C004057
:0C5B840082A0FFFF8290FFFFC4110020F0
:105B900070B5634B19684A1C1A60012800D1B9E03E
:105BA0000A788B1C5E4C2360022800D1B4E04D784B
:105BB000CB1C2360032800D1B0E08E780B1D23603E
:105BC0000438C0B2931E0D2B00D9A4E0052A32D0B0
:105BD0000F2A30D013000C3B012B3DD904231400B5
:105BE0009C43022C5AD0C978072A7AD84D4B002200
:105BF0001A704D4B1A68541C1C6015701A684B4B78
:105C00001B689A4269D0484B1A68541C1C60167075
:105C10001A68464B1B689A4278D0434B1A68541C4A
:105C20001C6011701A68414B1B689A4273D13E4B3D
:105C30003F4A1A606FE03B4B00221A703A4B1A68D9
:105C4000511C196015701A68384B1B689A4262D152
:105C5000354B374A1A605EE0324B1B78AB420BD0B3
:105C6000314B1A68511C196015701A682F4B1B684C
:105C70009A420FD02B4B1D702B4B1A68511C196088
:105C800016701A68294B1B689A4244D1264B284A41
:105C90001A6040E0244B264A1A60EBE7214B0022B1
:105CA0001A70214B1A68511C196015701A681F4B25
:105CB0001B689A420DD01C4B1A68511C1960167053
:105CC0001A681A4B1B689A4225D1174B184A1A605A
:105CD00021E0154B164A1A60EDE7134B144A1A607F
:105CE00091E7104B1B78AB428DD00F4B1A68541CB8
:105CF0001C6015701A680D4B1B689A4202D0094B44
:105D00001D7080E7084B0A4A1A60F8E7064B084AFC
:105D10001A6082E7002070BD0020FCE70020FAE74F
:105D2000801400209215002028150020FC0100207E
:045D3000C41100207A
:105D340070B582B0404B1B881BB2002B11DB3F4B6C
:105D44003F4A1A603F4B1B6818783F4B1B685A0048
:105D5400D21890423FD940283DD83C4D374C2600BC
:105D640025E0354A13883A490B401380E7E7FFF7EB
:105D74000DFF14E0374B02221A600BE0364B1A6811
:105D8400511C19603168097811701A68334B1B680B
:105D94009A421CD02368013323600138C0B22A4BD5
:105DA4001B685A00D218904215D9402813D8012BE9
:105DB400DDD02B68022BE1D0204B1B681B78022B13
:105DC400D8D0042BDAD1234B04221A60E2E7224B09
:105DD400234A1A60DEE7234B1A681F4B1B689A425A
:105DE40020D99B1AC4339BB201AA13801E4B0022F4
:105DF4001A6001AB1B889BB27E2B18D80E4B1B88F4
:105E04009BB26A46D380D3889B0402D40A4B174AB8
:105E14001A806B4606331B88DB040BD4064B144AEA
:105E24001A8007E09B1A9BB201AA1380DEE70E4B8F
:105E3400FF321A6002B070BD085C0040801400207C
:105E440000620040301500208414002064150020F6
:105E54008F0F0000A414002028150020FC0100204E
:105E6400C4110020241500207814002082A0FFFF14
:045E74008290FFFF1A
:105E780000B585B0234B1A6801921B681B0429D50D
:105E8800019A0F2313400393019A1023134002939E
:105E9800039B012B0BD0039B022B0BD0039B002BE6
:105EA8000ED1029B002B08D1FFF7E6FA1DE0FFF7A1
:105EB80053FD1AE0FFF73AFF17E0FFF75DFB14E028
:105EC800039B032B11D1104B1B68002B0DD1FFF73F
:105ED800D7FD0AE00B4B1B685B0508D4094B1B6810
:105EE8001B050AD5074B094A1A6005B000BDFFF724
:105EF800D7F8044B064A1A60F7E7024B054A1A60BE
:105F0800F3E7C046445C004084140020FFF7FFFF1D
:085F1800FFFBFFFF7F8000008A
:105F200070B5134B1B68002B21D0124B1A68511C03
:105F3000196010701A68104B1B689A4204D00F4EFB
:105F40000C4DAC24A4000AE00A4B0D4A1A60F6E797
:105F5000C02189008C466344991AA14207D9FAF7F7
:105F6000FBFA32682B68991A9A42F6D9F0E770BDAD
:105F70008814002020150020F80100201C150020A6
:045F8000F80D0020F8
:105F840000B5C54A13780133DBB2137042B2002A5C
:105F940023DBC24B1B78002B00D1A2E0C04B1B7843
:105FA4000F2219009143BF4A1278002A00D0BCE0A6
:105FB400BD4A1070BD4A00201070022218009043A0
:105FC4000200F12800D195E01F229343C02B00D199
:105FD4009DE0B44BFF221A708BE0F72800D139E121
:105FE400AD4B01221A70F0281BD0AD4B1870F3286A
:105FF40062D903000C33DBB2012B68D9FD2866D0CB
:10600400AB4B05221A700023A74A1370A74A1370DA
:10601400A24A1370A34A1370A64A1370A64A1370B7
:10602400D1E09F4BEF321A709C4B0F321A70002351
:106034009C4A13709F4A13709F4A137059E09C4BFB
:1060440005221A70964BF2321A700023964A137086
:10605400964A1370914A1370924A1370954A1370BA
:10606400954B1B78002B03D0934B00221A70AAE0A7
:106074000023894A1370904A13703AE08C4B06222D
:106084001A70894B1978864A1170F7221A70002306
:10609400864A1370814A1370824A1370854A1370BA
:1060A400854A13708FE0844B1B78002B00D0DFE00F
:1060B4007E4BF0321A70E4E0784BFF221A70002312
:1060C400784A13707B4A13707B4A137011E00023E3
:1060D400724A1370734A1370764A1370764A1370B7
:1060E40007E06D4A13706F4A1370724A1370724A54
:1060F400137000BD6E4BEF3A1A700023674A137099
:10610400684A13706B4A13706B4A13705BE0090999
:10611400674B1970614BE0321A700023614A1370A7
:10612400644A1370644A13704DE0624A1278002A7C
:1061340034D15E4A1070604A1278002A0FD1F22BD3
:1061440011D0F02B1CD00909594B1970534BFF2265
:106154001A700023534A1370564A137033E0554B98
:10616400FF221A70C5E7524B03221A7000234B4AD0
:1061740013704C4A13704F4A13704F4A137022E045
:106184004B4B04221A70FF234B4A1370434A13707B
:106194000023444A1370474A137014E0424A1178AA
:1061A4003F4B1970414B197811701870404B042201
:1061B4001A70FF23404A1370384A13700023394A77
:1061C40013703C4A13703D4B1B68002B00D190E7C1
:1061D4003B4B1A68531C364909781170394A1268C6
:1061E4009A422FD05A1C2E4909781970354B1B68D6
:1061F400934229D0531C2C4909781170314A1268F2
:106204009A4223D05A1C2949097819702D4B1B68CE
:1062140093421DD02A4B1A6000231F4A1370214A4F
:106224001370244A1370224B1B78072B01D8042BBC
:1062340004D11B4B1B78F02B00D85AE7174B0022D4
:106244001A7056E7204BCDE71F4AD3E71E4BD9E718
:106254001D4ADFE7012B00D1F1E6022B00D10DE747
:10626400134B07221A700E4B1B78F02B00D11AE740
:106274000D4A11780A4B19700C4B19781170F722DA
:106284001A700023054A1370064A1370094A1370E2
:10629400094A137097E7C046F910002096150020AC
:1062A400971500209B1500209915002098150020B3
:1062B400951500209A1500208912002088140020CA
:0C62C40020150020F8010020F80D00203B
:1062D000074B1B68002B00DBFEE7054A1168802393
:1062E0001B060B4313608369023383617047C0460A
:0462F0002CED00E0B1
:1062F40043466F72746820666F722053544D333274
:106304004630343220762E00202863293230323051
:106314002D323420572E536368656D6D6572740099
:08632400202D3E4442472000F9
:08632C004B65726E656C3A00CE
:106334004C330008A2330008FC330008FC33000887
:10634400B4330008C6330008D8330008EA33000821
:1063540020636F6E6669726D20772E75707065723A
:106364002063617365202759270000002063616E54
:0863740063656C6C6564200098
:10637C00205761726E3A2077696C6C206F7665726B
:10638C0072696465204B65726E656C204F50207786
:0C639C002E73616D65206E616D65200040
:1063A800426175642052617465206368616E676537
:1063B8007320696D6D6564696174656C792120006D
:1063C800656E746572204F4E4C592046495253549D
:0C63D80020322044494749545321200042
:1063E400536176652061637475616C20776F726B9D
:0C63F40020696E20466C617368203F0039
:10640000313238205352414D2062797465732073C4
:1064100074617274696E672066726F6D20307800E7
:10642000000000000000000000000000000000006C
:10643000000000000000000000000000000000005C
:10644000000000000000000000000000000000004C
:10645000000000000000000000000000000000003C
:10646000000000000000000000000000000000002C
:10647000000000000000000000000000000000001C
:10648000000000000000000000000000000000000C
:1064900000000000000000000000000000000000FC
:1064A00000000000000000000000000000000100EB
:1064B00000000500000000000000000000000000D7
:1064C00000000000000000000000000000000000CC
:1064D00000000000000001000000040000000400B3
:1064E00000000000000000000000000000000000AC
:1064F000000001000000000000000000000000009B
:10650000000000000000000000000000000000008B
:10651000000000000000000000000000000000007B
:106520000000000000000400000000000000050062
:106530000000050000000500000004000000040049
:106540000000040000000400000000000000010042
:106550000000010000000100000001000000030035
:10656000000003000000030000000300000003001F
:10657000000003000000030000000300000003000F
:106580000000030000000300000003000000020000
:1065900000000200000002000000020000000200F3
:1065A00000000100000001000000080000000800D9
:1065B00000000800000008000000080000000800BB
:1065C00000000800000008000000080000000800AB
:1065D000000008000000080000000800000008009B
:1065E0000000080000000800000008000000020091
:1065F0000000020000000100000001000000010096
:106600000000010000000100000005000000010082
:046610000000010085
:106614004552524F5200000044524F5000000000B7
:106624004455500000000000535741500000000042
:106634004F56455200000000524F54000000000025
:106644002D524F54000000005049434B00000000FD
:10665400524F4C4C00000000494E4A454354000040
:106664002B00000000000000312B0000000000009F
:106674002D00000000000000312D0000000000008B
:1066840041425300000000005348494654000000B2
:10669400414E4400000000004F5200000000000082
:1066A400584F5200000000004E4F540000000000FC
:1066B4002B2F2D00000000002A0000000000000025
:1066C4002F000000000000002A2F0000000000003E
:1066D4004D4F4400000000002F4D4F4400000000C7
:1066E40052414E444F4D00003D3D0000000000006B
:1066F400213D0000000000003E00000000000000FA
:106704003E3D0000000000003C00000000000000CE
:10671400553C0000000000003E3D00000000000069
:10672400303D000000000000564152434F4E00002F
:106734005245560000000000570000000000000011
:1067440052000000000000004B45593F00000000CB
:106754004B45590000000000454D4954000000001D
:106764002E000000000000002E4800000000000081
:106774002E440000000000002E2200000000000053
:10678400445A0000000000004858000000000000C7
:1067940052583F0000000000525800000000000062
:1067A40054580000000000004E545800000000003F
:1067B4005458220000000000584E4F5000000000C2
:1067C4004D5300000000000044530000000000008E
:1067D400544958000000000054494D450000000091
:1067E4004F480000000000004F4C00000000000073
:1067F40049505500000000004950440000000000CA
:10680400495A0000000000005244494E00000000B4
:1068140052414443000000002E53000000000000D9
:1068240046530000000000004F50530000000000D9
:106834005553455200000000534545000000000038
:106844004D454D00000000005354000000000000BE
:1068540052554E00000000004E4F2D4442470000A8
:106864004445425547000000464F524745540000F6
:1068740041424F52540000005245504C41434500A0
:10688400524553544F524500494600000000000051
:1068940043415345000000003C4341534500000080
:1068A4003E43415345000000454C53450000000061
:1068B4005448454E00000000444F00000000000012
:1068C400554E54494C0000005748494C45000000BF
:1068D400414741494E000000464F5200000000006D
:1068E4004C4F4F5000000000490000000000000021
:1068F400434F4E5449000000425245414B000000B2
:106904005A425245414B000052455455524E0000E4
:106914003A000000000000003B00000000000000FE
:10692400646F535452000000646F494F5354520033
:10693400646F4C4954000000646F4C495438420061
:10694400646F56414C554500646F52455600000033
:10695400646F494600000000646F434153450000E2
:10696400646F3C4341534500646F3E4341534500CB
:10697400646F454C53450000646F444F00000000B1
:10698400646F554E54494C00646F5748494C450058
:10699400646F414741494E00646F464F5200000006
:1069A400646F4C4F4F50000052502D3100000000D6
:1069B40052502D34000000004155544F45584500B5
:1069C40042415544000000004348414E4E454C00AE
:1069D40053504C4954000000564944504944000067
:1069E4003F00000000000000534156450000000035
:0869F4004C4F4144000000007B
:0469FC000403090483
:106A00001803430046006F007200740068002D00F8
:086A10004D004900440049005B
:106A1800FEE7FEE7FEE7FEE7FEE7FEE7FEE7FEE746
:106A2800FEE7FEE7FEE7FEE7FEE7FEE7FEE7FEE736
:106A3800FEE7FEE7FEE7FEE7FEE7FEE7FEE7FEE726
:106A4800FEE7FEE7FEE7FEE7FEE7FEE7FEE7FEE716
:106A5800FEE7FEE7FEE7FEE7FEE7FEE7FEE7FEE706
:106A6800FEE703488546FEF76DFA03E0704700002D
:046A780000180020E2
:106A7C0011488546114C20680434004201D08047EF
:106A8C00F9E70F480F49091A082903DB00220260B5
:106A9C00043001600C480D49884205D0026804306E
:106AAC0003B4904703BCF7E700208646EC46002071
:106ABC000021074A9047FEE7001800207C7100086F
:106ACC00A0150020E81600204D6E00084D6E000841
:046ADC008D0C000815
:106AE00004207146084202D1EFF3088001E0EFF381
:0C6AF0000980014908470000D16200083D
:106AFC002030204348414E4E454C20616363657005
:106B0C00747320414E59204D494449206368616E8D
:106B1C006E656C20696E20726563656976656420AC
:066B2C006D736773200089
:106B320010B5441C0078002806D0F9F766FB013432
:0A6B4200631E18780028F8D110BD7A
:106B4C00756E646572666C6F77212000202D2D2D7B
:026B5C00200017
:106B5E0010B5040003061B0F18003030392801D978
:106B6E0037331800F9F74BFB0F200440200030306C
:106B7E00392800D90730F9F742FB2020F9F73FFBFF
:026B8E0010BD38
:066B90002849502D3E00D3
:0E6B960010B5F9F77EFF2020F9F735FB10BD92
:106BA40063616E277420534545204B65726E656C96
:106BB4004F707300557365724865616465725F5305
:106BC40074727563743D0000566172436F6E3A5679
:066BD400616C75653D00D7
:106BDA002F280FD90300303BDBB2092B08D90A2929
:106BEA000BD00300413B052B0AD83738C0B2704797
:106BFA001800FCE701204042F9E701204042F6E78D
:066C0A0001204042F3E707
:106C10004572726F722300002028636F6C200000A1
:106C2000206E6F7420666F756E6400005F53796E1E
:106C300074617820457272005F537461636B204504
:106C4000727200005F436F6D70696C65206F6E6CCF
:106C5000790000005F4E6F20492F4F20436F6D6D0C
:106C600020416363657373005F496E76616C69648C
:106C700020436F64652061636365737300000000E7
:106C80005F6F7574206F6620436F6E746578740053
:106C90005F52756E74696D65206F6E6C79000000CF
:106CA0005F5468726561642063616E63656C6C65D6
:106CB000640000005F4E756D626572206F75742010
:106CC0006F662052616E6765000000005F44697660
:106CD0002E6279205A65726F000000002020636FD9
:0A6CE0006D70696C696E672E2E005E
:0A6CEA0010B50120FBF757FF10BDA5
:0A6CF40042617564526174653D0051
:0A6CFE0010B50020FBF74DFF10BD9C
:106D0800537461636B3D00002052657475726E00A8
:106D180020557365723D000020436F6465546872A6
:106D28006561643D00000000456D707479000000E5
:106D3800466C6173680000005F50726F6A65637427
:106D4800206C6F61646564002020204155544F45D4
:106D580058453D005465726D696E616C5F53706C87
:0E6D680069743D0020204D69646943683D0058
:0E6D760010B56820FBF717FCFCF755FB10BDAD
:106D8400555342205465726D696E616C5F436F6D3B
:106D94002077696C6C20676574206C6F73742100B4
:106DA4005553415254205465726D696E616C5F4352
:106DB4006F6D2077696C6C20676574206C6F7374D9
:026DC4002100AC
:0E6DC60010B56920FBF7EFFBFCF72DFB10BDAD
:106DD4001201000200000040830440572405000013
:026DE4000001AC
:0E6DE60010B56A20FBF7DFFBFCF71DFB10BDAC
:026DF40000009D
:0E6DF60010B56B20FBF7D7FBFCF715FB10BDAB
:106E0400120368006F006D0065006D00610064008E
:026E1400650017
:0E6E160010B56E20FBF7C7FBFCF719FB10BD93
:106E240012010002000000408304435724050201BC
:026E340000015B
:0E6E360010B56F20FBF7B7FBFCF709FB10BD92
:096E440028566172436F6E3D0097
:0E6E4E0010B57020FBF7ABFBFCF7FDFA10BD92
:106E5C00203C2D6E6F742061204B65726E656C202A
:106E6C004F50206E6F722061206E756D62657200DE
:106E7C00203C2D696E76616C696420666F722042CD
:106E8C0061636B2D4374726C00000000203C2D522A
:0D6E9C00756E74696D65204572726F72002D
:0A6EAA0010B50120FDF731FB10BD0B
:106EB40020202841444320696E6974292000000081
:0D6EC400202028414443206F6666292000ED
:0A6ED20010B50020FDF71DFB10BDF8
:106EDC002064656275672066696E697368656420F5
:016EEC0000A5
:106EEE000A0010D00300400800E052008242FCD994
:106EFE00002000E05208934200D39B1A40418A4280
:0A6F0E00F8D1190070470020704709
:106F18004C6F616420466C6173682050726F6A65BB
:106F28006374203F000000004C6F616420456D7061
:0D6F380074792050726F6A656374203F0009
:106F46008446002A05D00B78037001300131013ADE
:066F5600F9D1604670470E
:106F5C00555342206173207669727475616C2043BD
:106F6C004F4D3D00555342206173204D49444920FB
:0B6F7C00696E746572666163653D001C
:076F88006E6F20555342001B
:0F6F9000564944203D200000504944203D200038
:106FA00009024300020100803109040000010202CD
:106FB0000000052400100105240103000424020739
:106FC00005240600010705830310004009040100A1
:106FD000020A0000000705810240000007050202C6
:036FE0004000006E
:076FE40000C20100000008DB
:106FEC000902650002010080310904000000010162
:106FFC00000009240100010900010109040100023B
:10700C0001030000072401000141000624020101D4
:10701C0000062402020200092403010301020100FC
:10702C00092403020401010100090581024000004A
:10703C0000000525010103090502024000000000C3
:05704C00052501010112
:1070520010B50400000F16D12001000F17D1200235
:10706200000F18D12003000F19D12004000F1AD1EC
:107072002005000F1BD12006000F1CD10F2020403D
:10708200F9F7B9F910BDF9F7B6F92001000FF9F7D0
:10709200B2F92002000FF9F7AEF92003000FF9F759
:1070A200AAF92004000FF9F7A6F92005000FF9F755
:0C70B200A2F92006000FF9F79EF9DFE7B5
:1070BE0010B504003020F9F7A2F87820F9F79FF800
:0870CE002000FFF7BFFF10BD19
:1070D600CA1751408B1A17D0C1174A4004B448400A
:1070E600411A48081A0000E052008242FCD90020EA
:1070F60000E05208914200D3891A40419A42F8D1E1
:0C71060004BC5040801A70470020704705
:107112000A000FD00300400800E052008242FCD96E
:10712200002000E05208934200D39B1A40418A4259
:08713200F8D1704700207047FE
:10713A00CA1751408B1A19D0C11706B44840411AD0
:10714A0048081A0000E052008242FCD9002000E000
:10715A005208914200D3891A40419A42F8D10CBC94
:10716A0053405840C01A5140891A7047002070474E
:10717C00A57300080802002098130000BB730008D8
:10718C00000000209C7100080802000000000000B4
:10719C00AD110008BD110008E5110008151200081A
:1071AC002D1200084112000865120008891200080F
:1071BC00C91200082913000889130008A513000838
:1071CC00B5130008D1130008E1130008F9130008E7
:1071DC00411400085D140008791400089514000887
:1071EC00A5140008B5140008D114000809150008EE
:1071FC004115000879150008B9150008D1150008CB
:10720C00F115000825160008491600086D1600082F
:10721C0091160008B116000811160008094A00085A
:10722C00D94D0008D516000815170008B92A000812
:10723C00C51C0008211C0008211D0008691D000840
:10724C00511F0008EB6C000849170008691700086B
:10725C00152D0008B12E0008691F0008811F0008B9
:10726C00FF6C0008891700085D2F00088D2F00089F
:10727C00B1170008CD170008F52F00086130000881
:10728C00CD3000082D31000889310008D1310008BB
:10729C00C9320008891D0008E9180008BD1F000844
:1072AC004D1E0008953B0008814E00080919000886
:1072BC001519000821190008391C0008253F000881
:1072CC009D3F000839440008C5440008776D00084C
:1072DC00C76D0008E76D0008F76D000891270008DE
:1072EC00ED170008D9270008176E0008376E000844
:1072FC004F6E0008052800083128000821180008E6
:10730C00691A00083D18000851180008791800087F
:10731C00514A000889280008AB6E0008D36E00089B
:10732C002D1900086D1900088D190008B9190008ED
:10733C0079450008A5450008D54500080546000814
:10734C00E5190008091A0008991A0008D11A000852
:10735C00391A0008091B0008591B0008011C0008F9
:10736C00111C000855250008954A0008711C0008DE
:10737C00554B0008654C0008C9460008DD4C000858
:10738C00194D000801000000F810002088120020A0
:08739C00C0110020006CDC02AE
:1073A400206861680834094204D000220270013068
:0673B4000139FBD1704716
:1073BA0020686168A2680C34124205D00B78037009
:0A73CA0001300131013AF9D170479A
:0400000508006A6B1A
:00000001FF
